S00F0000746563776172652E737265632A
S315080028000000012075C800084D5100084F51000806
S3150800281051510008535100085551000800000000A6
S3150800282000000000000000000000000061C300086E
S31508002830575100080000000001C40008595100085B
S31508002840C5C80008C5C80008C5C80008C5C8000826
S31508002850C5C80008C5C80008C5C80008C5C8000816
S31508002860C5C80008C5C80008C5C80008C5C8000806
S315080028707151000881510008C5C80008C5C800087C
S31508002880C5C80008C5C8000891510008A15100082C
S31508002890B1510008C1510008D1510008C5C8000847
S315080028A0C5C80008C5C80008C5C80008C5C80008C6
S315080028B0C5C800080000000000000000C5C80008E0
S315080028C0C5C800080000000000000000E15100082B
S315080028D000000000C5C80008C5C8000800000000C0
S315080028E0C5C80008C5C800080000000000000000B0
S315080028F000000000000000000000000000000000CA
S31508002900000000000000000000000000C5C8000824
S315080029100000000000000000C5C80008C5C800087F
S31508002920C5C80008C5C80008F1510008C5C8000890
S31508002930C5C80008000000000000000000000000F4
S31508002940C5C80008C5C80008C5C80008C5C8000825
S31508002950C5C80008C5C80008C5C80008C5C8000815
S31508002960C5C80008C5C80008C5C80008000000009A
S31508002970C5C80008C5C8000800000000000000001F
S31508002980C5C80008C5C80008C5C800082255AAEE6B
S3150800299010B5054C237833B9044B13B10448AFF38B
S315080029A000800123237010BD1801002000000000DC
S315080029B098CA000808B5034B1BB103490348AFF38F
S315080029C0008008BD000000001C01002098CA00080D
S315080029D081F0004102E000BF83F0004330B54FEAC2
S315080029E041044FEA430594EA050F08BF90EA020F2F
S315080029F01FBF54EA000C55EA020C7FEA645C7FEAC2
S31508002A00655C00F0E2804FEA5454D4EB5555B8BFE4
S31508002A106D420CDD2C4480EA020281EA030382EA55
S31508002A20000083EA010180EA020281EA0303362DE7
S31508002A3088BF30BD11F0004F4FEA01314FF4801CBA
S31508002A404CEA113102D0404261EB410113F0004FCC
S31508002A504FEA03334CEA133302D0524263EB430383
S31508002A6094EA050F00F0A780A4F10104D5F1200E21
S31508002A700DDB02FA0EFC22FA05F2801841F100017C
S31508002A8003FA0EF2801843FA05F359410EE0A5F150
S31508002A9020050EF1200E012A03FA0EFC28BF4CF081
S31508002AA0020C43FA05F3C01851EBE37101F0004537
S31508002AB007D54FF0000EDCF1000C7EEB00006EEB44
S31508002AC00101B1F5801F1BD3B1F5001F0CD34908CE
S31508002AD05FEA30004FEA3C0C04F101044FEA445225
S31508002AE012F5800F80F09A80BCF1004F08BF5FEAAC
S31508002AF0500C50F1000041EB045141EA050130BD8C
S31508002B005FEA4C0C404141EB0101013C28BFB1F59D
S31508002B10801FE9D291F0000F04BF01460020B1FAE8
S31508002B2081F308BF2033A3F10B03B3F120020CDABB
S31508002B300C3208DD02F1140CC2F10C0201FA0CF099
S31508002B4021FA02F10CE002F11402D8BFC2F1200CFE
S31508002B5001FA02F120FA0CFCDCBF41EA0C019040B4
S31508002B60E41AA2BF01EB0451294330BD6FEA0404FD
S31508002B701F3C1CDA0C340EDC04F11404C4F12002E8
S31508002B8020FA04F001FA02F340EA030021FA04F3FA
S31508002B9045EA030130BDC4F10C04C4F1200220FA51
S31508002BA002F001FA04F340EA0300294630BD21FA8F
S31508002BB004F0294630BD94F0000F83F4801306BF55
S31508002BC081F480110134013D4EE77FEA645C18BF49
S31508002BD07FEA655C29D094EA050F08BF90EA020FE0
S31508002BE005D054EA000C04BF1946104630BD91EAD8
S31508002BF0030F1EBF0021002030BD5FEA545C05D1DB
S31508002C004000494128BF41F0004130BD14F5800419
S31508002C103CBF01F5801130BD01F0004545F0FE418D
S31508002C2041F470014FF0000030BD7FEA645C1ABFC2
S31508002C30194610467FEA655C1CBF0B46024650EAF9
S31508002C40013406BF52EA033591EA030F41F4002125
S31508002C5030BD00BF90F0000F04BF0021704730B5AB
S31508002C604FF4806404F132044FF000054FF0000180
S31508002C7050E700BF90F0000F04BF0021704730B541
S31508002C804FF4806404F1320410F0004548BF404216
S31508002C904FF000013EE700BF42004FEAE2014FEA6B
S31508002CA031014FEA02701FBF12F07F4393F07F4F46
S31508002CB081F06051704732F07F4208BF704793F049
S31508002CC07F4F04BF41F40021704730B54FF460745C
S31508002CD001F0004521F000411CE700BF50EA01025F
S31508002CE008BF704730B54FF000050AE050EA010208
S31508002CF008BF704730B511F0004502D5404261EB78
S31508002D0041014FF4806404F132045FEA915C3FF4B8
S31508002D10D8AE4FF003025FEADC0C18BF03325FEA55
S31508002D20DC0C18BF033202EBDC02C2F1200300FA06
S31508002D3003FC20FA02F001FA03FE40EA0E0021FA2B
S31508002D4002F11444BDE600BF70B54FF0FF0C4CF419
S31508002D50E06C1CEA11541DBF1CEA135594EA0C0FCB
S31508002D6095EA0C0F00F0DEF82C4481EA030621EA06
S31508002D704C5123EA4C5350EA013518BF52EA033541
S31508002D8041F4801143F4801338D0A0FB02CE4FF0F3
S31508002D900005E1FB02E506F00042E0FB03E54FF023
S31508002DA00006E1FB03569CF0000F18BF4EF0010E1B
S31508002DB0A4F1FF04B6F5007F64F5407404D25FEA17
S31508002DC04E0E6D4146EB060642EAC62141EA5551CA
S31508002DD04FEAC52040EA5E504FEACE2EB4F1FD0C0C
S31508002DE088BFBCF5E06F1ED8BEF1004F08BF5FEA8A
S31508002DF0500E50F1000041EB045170BD06F000463C
S31508002E0046EA010140EA020081EA0301B4EB5C04E8
S31508002E10C2BFD4EB0C0541EA045170BD41F48011E0
S31508002E204FF0000E013C00F3AB8014F1360FDEBF05
S31508002E30002001F0004170BDC4F10004203C35DAE1
S31508002E400C341BDC04F11404C4F1200500FA05F364
S31508002E5020FA04F001FA05F240EA020001F0004205
S31508002E6021F0004110EBD37021FA04F642EB06017B
S31508002E705EEA430E08BF20EAD37070BDC4F10C04A5
S31508002E80C4F1200500FA04F320FA05F001FA04F269
S31508002E9040EA020001F0004110EBD37041F1000155
S31508002EA05EEA430E08BF20EAD37070BDC4F1200560
S31508002EB000FA05F24EEA020E20FA04F301FA05F2C8
S31508002EC043EA020321FA04F001F0004121FA04F270
S31508002ED020EA020000EBD3705EEA430E08BF20EA40
S31508002EE0D37070BD94F0000F0FD101F0004640007A
S31508002EF041EB010111F4801F08BF013CF7D041EAFC
S31508002F00060195F0000F18BF704703F000465200FF
S31508002F1043EB030313F4801F08BF013DF7D043EAD0
S31508002F200603704794EA0C0F0CEA135518BF95EA86
S31508002F300C0F0CD050EA410618BF52EA4306D1D10D
S31508002F4081EA030101F000414FF0000070BD50EA2C
S31508002F50410606BF1046194652EA430619D094EAB6
S31508002F600C0F02D150EA013613D195EA0C0F05D1A0
S31508002F7052EA03361CBF104619460AD181EA0301F4
S31508002F8001F0004141F0FE4141F470014FF00000AC
S31508002F9070BD41F0FE4141F4780170BD70B54FF047
S31508002FA0FF0C4CF4E06C1CEA11541DBF1CEA1355C7
S31508002FB094EA0C0F95EA0C0F00F0A7F8A4EB0504A9
S31508002FC081EA030E52EA03354FEA013100F08880A0
S31508002FD04FEA03334FF0805545EA131343EA126369
S31508002FE04FEA022245EA111545EA10654FEA00261E
S31508002FF00EF000419D4208BF964244F1FD0404F5D7
S31508003000407402D25B084FEA3202B61A65EB030532
S315080030105B084FEA32024FF480104FF4002CB6EBEF
S31508003020020E75EB030E22BFB61A754640EA0C006F
S315080030305B084FEA3202B6EB020E75EB030E22BFAF
S31508003040B61A754640EA5C005B084FEA3202B6EBF0
S31508003050020E75EB030E22BFB61A754640EA9C00AF
S315080030605B084FEA3202B6EB020E75EB030E22BF7F
S31508003070B61A754640EADC0055EA060E18D04FEA3D
S31508003080051545EA16754FEA06164FEAC30343EADD
S3150800309052734FEAC2025FEA1C1CC0D111F4801FAA
S315080030A00BD141EA00014FF000004FF0004CB6E7A3
S315080030B011F4801F04BF01430020B4F1FD0C88BF42
S315080030C0BCF5E06F3FF6AFAEB5EB030C04BFB6EB4D
S315080030D0020C5FEA500C50F1000041EB045170BD40
S315080030E00EF0004E4EEA113114EB5C04C2BFD4EB6D
S315080030F00C0541EA045170BD41F480114FF0000EF1
S31508003100013C90E645EA060E8DE60CEA135594EA6C
S315080031100C0F08BF95EA0C0F3FF43BAF94EA0C0F6F
S315080031200AD150EA01347FF434AF95EA0C0F7FF4E4
S3150800313025AF104619462CE795EA0C0F06D152EA38
S3150800314003353FF4FDAE1046194622E750EA41061C
S3150800315018BF52EA43067FF4C5AE50EA41047FF42D
S315080031600DAF52EA43057FF4EBAE12E74FF0FF3C92
S3150800317006E000BF4FF0010C02E000BF4FF0010C63
S315080031804DF804CD4FEA410C7FEA6C5C4FEA430CDC
S3150800319018BF7FEA6C5C1BD001B050EA410C0CBF2B
S315080031A052EA430C91EA030F02BF90EA020F00208D
S315080031B0704710F1000F91EA030F58BF994208BFF4
S315080031C090422CBFD8176FEAE37040F001007047B1
S315080031D04FEA410C7FEA6C5C02D150EA013C07D108
S315080031E04FEA430C7FEA6C5CD6D152EA033CD3D053
S315080031F05DF8040B704700BF8446104662468C464D
S315080032001946634600E000BF01B5FFF7B7FF00287F
S3150800321048BF10F1000F01BD4DF808EDFFF7F4FFA8
S315080032200CBF012000205DF808FB00BF4DF808ED33
S31508003230FFF7EAFF34BF012000205DF808FB00BF56
S315080032404DF808EDFFF7E0FF94BF012000205DF878
S3150800325008FB00BF4DF808EDFFF7CEFF94BF01202D
S3150800326000205DF808FB00BF4DF808EDFFF7C4FF26
S3150800327034BF012000205DF808FB00BF4FEA410279
S31508003280B2F1E04324BFB3F5001CDCF1FE5C0DD9B6
S3150800329001F0004C4FEAC0024CEA5070B2F1004F00
S315080032A040EB830008BF20F00100704711F0804F03
S315080032B021D113F13872BCBF01F00040704741F4C8
S315080032C080114FEA5252C2F11802C2F1200C10FACC
S315080032D00CF320FA02F018BF40F001004FEAC123B0
S315080032E04FEAD32303FA0CFC40EA0C0023FA02F354
S315080032F04FEA4303CCE77FEA625307D150EA01332A
S315080033001EBF4FF0FE4040F44000704701F00040F9
S3150800331040F0FE4040F40000704700BF08B501F0D9
S31508003320CDF800F0010401F09BFA044000F0CEFB52
S31508003330044001F02DF8044000F01AFE044000F0A5
S315080033406BFE044001F0CEF8044000F06FFC044028
S3150800335001F030FA044000F061FF044000F09EF9E5
S31508003360044000F0F9F804421AD106F069FC02207C
S3150800337001F098F80D4B1B689B0B642202FB03F3C4
S31508003380002BF4D000BF00BF00BF00BF00BF00BFC6
S3150800339000BF00BF00BF00BF00BF00BF013BEFE793
S315080033A0034B186806F0BFFCFEE700BF9400002038
S315080033B03401002008B5054A0021054806F055FCE9
S315080033C0044B1860003818BF012008BDBCCA0008A5
S315080033D01D3300083401002000B585B0EC468CE8A2
S315080033E00F0000231A4661460548006806F0B9FE34
S315080033F00121044B186806F043FD05B05DF804FB8F
S31508003400440100204001002008B50146024B186817
S3150800341006F036FD08BD00BF4001002030B589B072
S315080034207FE000231A4602A94848006806F0DBFE3A
S315080034309DF808509DF81130012B11D0022B2FD082
S31508003440002B7BD1082D37D86AB2002A76D0013DE9
S31508003450072D73D8DFE805F0383C4072474C585BB7
S31508003460142D08D9FF228DF81820059A012106A8DF
S3150800347000F01CFF62E0284600F0F4FA01908DF88F
S31508003480185004220DF119010DEB020001F0DAFEC5
S315080034909DF81130059A052106A800F007FF4DE0B2
S315080034A004220DEB02010DF1090001F0CBFE019992
S315080034B0284600F083FA41E0FF2D3FD1002000F0B6
S315080034C0C5F803F067F939E0012000F0BFF835E0E8
S315080034D0002000F0BBF831E040F6B8311C4B186804
S315080034E006F092FC2AE00021132000F0ADFA25E050
S315080034F006228DF8182007228DF81920059A022130
S3150800350006A800F0D3FE19E000F0F2FA16E000F083
S315080035100FFB13E0022000F0C5FF12E0002000F0C8
S3150800352095F84FF0FF33002207210A48006806F095
S31508003530F4FC044610F0010F7FF473AF14F0020F89
S31508003540E8D114F0040FECD0E8E700BF44010020EE
S31508003550380100204001002070B52A4806F06EFCAC
S31508003560294B1860041E18BF0124284A0021284840
S3150800357006F07BFB274B186000280CBF002404F0DC
S315080035800104254A1021082006F0A0FD234B1860E7
S3150800359000280CBF002404F00104214D214B02220F
S315080035A00121284606F0DCFB1F4E306000280CBFC0
S315080035B0002404F001041D4B04220121284606F0CC
S315080035C0CFFB1B4D286000280CBF002404F0010423
S315080035D04FF47A71306806F017FC002814BF0024EF
S315080035E004F0010440F6B831286806F00DFC0028FE
S315080035F014BF002404F001040E4800F07FFE2046A4
S3150800360070BD00BF58CB00084001002080CB0008E1
S315080036101D3400084801002068CB0008440100203A
S315080036200934000848CB00083C01002038CB0008C4
S3150800363038010020D933000808B50146024B18683E
S3150800364006F01EFC08BD00BF4C01002010B504465C
S315080036500146032000F0EAFE2146122000F0F4F9A4
S3150800366010BD08B5122000F011FA08BD08B5F2EE33
S31508003670087AB4EEE70AF1EE10FA01DDB0EE670A51
S31508003680F9EE047AB4EEE70AF1EE10FA01D5B0EED7
S31508003690670A00F009FD00F0010008BD38B5174AB1
S315080036A00021174806F0E1FA164B1860041E18BFE9
S315080036B00124154806F0C2FB144B186000280CBFFD
S315080036C0002404F00104124B01221146114806F0A9
S315080036D047FB114D286000280CBF002404F00104A4
S315080036E09FED0E0AFFF7C2FFC821286806F08CFB7B
S315080036F0002814BF002004F0010038BDF8CB0008EC
S315080037002137000854010020D8CB00084C010020BE
S31508003710E8CB0008393600085001002000000000F8
S3150800372008B52DED0C8BDFED6B9AB0EE699AF0EECD
S31508003730698AB0EE698A3EE00020FFF787FF6BE0F2
S315080037409FED649AF4EEE7CAF1EE10FA02D57CEE24
S31508003750E76A01E0DFED5F6AB4EEC79AF1EE10FAA8
S3150800376007D4F4EEC76AF1EE10FA00F39180B0EED2
S31508003770479A3DEE0D7A78EEEAAA27EE2A7ADFED29
S31508003780566A6BEEA66A37EE267AF1EE479A79EE16
S31508003790277A77EEC77AF4EECC7AF1EE10FA06DCE1
S315080037A0F4EEEC7AF1EE10FA75D4B0EE67CAB0EE24
S315080037B04C0AFFF75BFFF0EE69BAB0EE49BAF0EED5
S315080037C068AAB0EE48AA4FF0FF3300220121434809
S315080037D0006806F0A2FB10F0010FF4D0404803F091
S315080037E0C8FEFFF73EFF9FED3B8AF0EE488AB0EE33
S315080037F0489AF0EE489A0028DDD0002000F046F9F5
S3150800380000284BD10E2000F045F9DFED367AB4EEEC
S31508003810E70AF1EE10FA8FDC022000F03BF9B0EE71
S31508003820409A032000F036F9F0EE409A042000F0A2
S3150800383031F9B0EE40DA062000F02CF9B0EE40CAB5
S31508003840072000F027F9F0EE40CA092000F022F917
S31508003850F0EE408A052000F01DF938EEC08A69EEC0
S31508003860087AB6EE007A29EE877ADFED1F6A27EE28
S31508003870267A3AEE08AA27EE0A7A37EE0B7AB4EEDB
S31508003880E7CAF1EE10FA7FF75BAF3CEE679A59E7A5
S31508003890B0EE669A6DE7B0EE6CCA88E7002000F0D5
S315080038A0F5F8012808D0F0EE6B9AB0EE4B9AF0EED8
S315080038B06A8AB0EE4A8A7EE700F0ECF8FFF7D6FE91
S315080038C0DFED049AB0EE699AF0EE698AB0EE698A7D
S315080038D071E700BF000000009A99193F4C010020CB
S315080038E0640300200000C842CDCC4C3E01288CBFA2
S315080038F00020012070470000084B03EB00139B686B
S315080039008B4207D8054B03EB0013DB688B4203D2C7
S3150800391000207047002070470120704738CC000807
S31508003920084B03EB00139B688B4207DC054B03EB44
S315080039300013DB688B4203DA0020704700207047CB
S315080039400120704738CC00080C4B03EB0013D3ED6D
S31508003950027AF4EEC07AF1EE10FA0BD8074B03EBB5
S315080039600013D3ED037AF4EEC07AF1EE10FA03DA17
S3150800397000207047002070470120704738CC0008A7
S3150800398008B503010C4AD35C13F0010F09D113F0F3
S31508003990020F0BD113F0040F0BD00846FFF7A6FF52
S315080039A003E000EE101AFFF7CFFF08BDFFF7B8FFD8
S315080039B0FBE7FFF7A1FFF8E738CC000838B50301A5
S315080039C00D4AD35C13F0080F00D038BD04460D46E7
S315080039D04FF0FF31094B186806F022FB29462046AE
S315080039E0FFF7CEFF10B1064B43F83450034B186867
S315080039F006F045FBE9E700BF38CC0008580100206F
S31508003A005C01002038B504460D464FF0FF310C4BDB
S31508003A10186806F005FB29462046FFF7B1FF30B9BE
S31508003A20084B03EBC4031A7942F002021A71054BDC
S31508003A3043F83450024B186806F021FB38BD00BF26
S31508003A40580100205C01002008B5FFF7DBFF08BD20
S31508003A5000B583B08DED010A0199FFF7D3FF03B0D6
S31508003A605DF804FB38B50446064D4FF0FF3128686B
S31508003A7006F0D6FA044B53F83440286806F0FFFAE5
S31508003A80204638BD580100205C01002008B5FFF724
S31508003A90E9FF08BD08B5FFF7E5FF00EE100A08BD07
S31508003AA008B5034B03EB00135968FFF7ABFF08BDD6
S31508003AB038CC000810B5002404E0E0B2FFF7F0FFA8
S31508003AC00134A4B2142CF8D910BD000010B506486C
S31508003AD006F05DFA054B1860041E18BF0124FFF7AF
S31508003AE0E9FF204610BD00BF28CC00085801002079
S31508003AF038B500F0A5FE00F00105002401E0013408
S31508003B00E4B2142C0ED82301084AD35C13F0100F24
S31508003B10F5D02046FFF7A6FF0146204600F063FED3
S31508003B200540ECE700F07EFE284038BD38CC00089A
S31508003B3030B583B00024012501E00134E4B2142C29
S31508003B4010D82301114AD35C13F0100FF5D001A940
S31508003B50204600F041FE0540EFD001992046FFF7C8
S31508003B6051FFEAE77DB103B030BD0134E4B2142C4D
S31508003B70F9D82301054AD35C13F0100FF5D0204677
S31508003B80FFF78EFFF1E70024F1E700BF38CC000805
S31508003B9008B572B10D4B60F07F00187000225A709C
S31508003BA099700B480323838100F0AAFC00F00100FA
S31508003BB008BD064B60F07F00187059700448022350
S31508003BC0838100F09DFC00F00100F1E70802002067
S31508003BD00000002010B50C4692B1114B1870002257
S31508003BE05A709A700F480323838100F089FC00F00D
S31508003BF001000D4B5A789B7843EA0223238010BDB7
S31508003C00074B187000225A7006480223838100F079
S31508003C1077FC00F00100044B5B782380EFE700BFD8
S31508003C2008020020000000201002002038B51448C1
S31508003C3006F0ADF9134D2860041E18BF01244FF095
S31508003C40FF3106F0EDF9002000F082FB0022822108
S31508003C501046FFF79DFF0440002000F089FB012075
S31508003C6000F076FB002282211046FFF791FF044000
S31508003C70012000F07DFB286806F001FA204638BDD1
S31508003C8094CD0008040200202DE9F04182B00F46C9
S31508003C90904600230B70ADF8063018B1012854D0B1
S31508003CA0012600E00126404D4FF0FF31286806F056
S31508003CB0B7F9304600F04CFB0022A0211046FFF76A
S31508003CC067FF00F00104304600F052FB286806F052
S31508003CD0D6F9642006F036F84FF0FF31286806F06A
S31508003CE09FF9304600F034FB01220DF1060110461B
S31508003CF0FFF770FF0440304600F03AFB286806F0EC
S31508003D00BEF924B3BDF8063013F0010F24D15B08C1
S31508003D10ADF80630A8F80030234D4FF0FF3128687B
S31508003D2006F07EF9304600F013FB00228421104687
S31508003D30FFF72EFF0440304600F01AFB286806F00D
S31508003D409EF9204602B0BDE8F0810026ABE73B7835
S31508003D5043F002033B70F4E7134C4FF0FF31206841
S31508003D6006F05EF9304600F0F3FA002239460720DD
S31508003D70FFF730FF304600F0FBFA304600F0E8FA6D
S31508003D80002282211046FFF703FF304600F0F0FAC2
S31508003D90206806F074F93B7803F0FC033B7043F0A7
S31508003DA001033B700024CCE7040200200000000059
S31508003DB0F0B585B0012005F0C5FF082262496348C1
S31508003DC001F0C0FF9EE004244FF0FF31604B1868F5
S31508003DD006F026F900230AE0E1185B4A32F81110CA
S31508003DE004AA02EB830242F8101C01339BB2032B90
S31508003DF0F2D91420FFF74EFE002325E004AA02EBB1
S31508003E00830252ED047AF8EE677A9FED527A67EEEE
S31508003E10877A9FED517A67EE877A67EE807A4F4AFE
S31508003E2002EB830292ED007A67EE277A4C4A02EBA0
S31508003E30830292ED007A77EEC77A4A4A02EB83024A
S31508003E40C2ED007A01339BB2032BD7D9002401E0D7
S31508003E500134A4B2032C1DD8424B03EB8403186823
S31508003E60FEF71AFF06460F4633A3D3E90023FFF7EA
S31508003E70F1F90028ECD032A3D3E9002330463946BD
S31508003E80FFF7D4F90028E3D0364B03EB840300226E
S31508003E901A60DDE7334C94ED020A0B20FFF7D8FDD4
S31508003EA094ED030A0C20FFF7D3FDD4ED037AF5EE63
S31508003EB0407AF1EE10FA36D19FED2B0A0D20FFF766
S31508003EC0C7FD284C94ED020AD4ED037A20EE270AA2
S31508003ED00E20FFF7BDFD94ED000A0F20FFF7B8FD91
S31508003EE094ED010A1020FFF7B3FD94ED000AD4ED16
S31508003EF0017A20EE270A1120FFF7AAFD144B18684D
S31508003F0006F0BDF84FF0FF3300220321174800687A
S31508003F1006F003F810F0020F7FF455AF10F0010F0A
S31508003F20F0D0002450E70F4B93ED020A80EE270AE3
S31508003F300D20FFF78DFDC4E79A9999999999A9BF1C
S31508003F409A9999999999A93F3402002070040020FA
S31508003F50280200200000803D0000803924CE000899
S31508003F6014CE000818020020000000002C020020D1
S31508003F7010B50F4A00210F4805F077FE0E4B186062
S31508003F80041E18BF01240D4805F058FF0C4B186095
S31508003F9000280CBF002404F001040A4805F0F7FFC6
S31508003FA0094B186000280CBF002004F0010010BD62
S31508003FB0F0CD0008B13D000830020020E0CD000831
S31508003FC02C020020D0CD00082802002008B50221C6
S31508003FD0024B186805F054FF08BD00BF2C020020EC
S31508003FE008B50121024B186805F04AFF08BD00BF55
S31508003FF02C020020836D836D836D836DC36CDB6B30
S315080040007047000008B50146024B186805F038FFEE
S3150800401008BD00BF4C02002038B51A4A00211A48CC
S3150800402005F023FE194B1860041E18BF0124184812
S3150800403005F004FF174B186000280CBF002404F095
S315080040400104154B01221146144805F089FE144D4A
S31508004050286000280CBF002404F001040021114840
S3150800406002F039FC002814BF002404F001043221B0
S31508004070286805F0C9FE002814BF002004F00100D6
S3150800408038BD00BF88CE0008F5410008540200205C
S3150800409068CE00084C02002078CE000805400008CB
S315080040A050020020C803002008B5064B83ED000A1D
S315080040B00121054B186805F0E3FEB0FA80F04009C7
S315080040C008BD00BF440200204C020020000000008A
S315080040D008B52DED028B10EE100AFEF7DDFD11A3D3
S315080040E0D3E90023FEF77AFC10A3D3E90023FEF7F1
S315080040F055FFFFF7C3F808EE100ADFED097A28EE38
S31508004100278A1420FFF7C6FCC8EE007AFCEEE77A89
S3150800411017EE900ABDEC028B08BD00BFAFF3008016
S3150800412000F07F454A0C022B87163440166BB8C838
S315080041303D0D41400000000008B52DED028B2A4BCD
S31508004140D3ED007A294B93ED008AF4EEC87AF1EEA6
S3150800415010FA26D517EE900AFEF79EFD20A3D3E99E
S315080041600023FEF73BFCFFF789F807EE900A1E4B83
S315080041701860B4EEE78AF1EE10FA01D583ED008AED
S31508004180194B93ED000AFFF7A3FF034600221146D9
S31508004190174802F0D2FBB0FA80F04009BDEC028B5A
S315080041A008BDF4EEC87AF1EE10FAE9DD17EE900ACA
S315080041B0FEF772FD0AA3D3E90023FEF70DFCFFF70D
S315080041C05DF807EE900A084B1860B4EEE78AF1EE40
S315080041D010FAD5DD83ED008AD2E700BFAFF3008081
S315080041E09A9999999999B93F480200204402002062
S315080041F0C803002008B54FF0FF3300220121064806
S31508004200006805F08AFE10F0010FF4D0FFF794FF5E
S31508004210002000F027F9EEE74C02002070B50420D4
S3150800422000F020F91D4C237803432370032000F087
S3150800423019F9237843EA40032370022000F012F9A3
S31508004240237843EA80032370012000F00BF92378D2
S3150800425043EAC000C0B22070114E336843EA4013E7
S315080042603360104D1049284601F00DFF04463146CB
S31508004270284601F008FF0443E4B2284601F086FF09
S315080042800443E4B20221284602F0C8F8204310F09D
S31508004290FF0F0CBF0120002070BD00BF5802002090
S315080042A044000020000400206C000020082901D9E1
S315080042B00020704700B587B012021FFA82FC4CEA4C
S315080042C003130C4A1278134343F410730093002324
S315080042D001930293039304918DF814300123024647
S315080042E06946054801F080FFB0FA80F0400907B03A
S315080042F05DF804FB5802002000040020014B1860FA
S31508004300704700BF5C02002030B58FB005AB07AA26
S31508004310002101F0DEFF079BC3F300220492C3F3DA
S3150800432001138DF80D309DF82C208DF80C2001AC6A
S31508004330214605A800F086FF034B1D6894E80F0088
S31508004340A8470FB030BD00BF5C02002070470000D0
S3150800435008B5064B4FEA401C03EB4010027F8188E4
S3150800436053F80C0003F00BF808BD00BFACCE0008EC
S3150800437008B5064B4FEA401C03EB4010027E8188C5
S3150800438053F80C0002F0FBFF08BD00BFACCE0008D6
S3150800439070B582B0224B1A6E42F001021A661B6E85
S315080043A003F001030193019B012500240BE0002380
S315080043B01D401C4B4A0103EB41110431985802F089
S315080043C0FFFE0134E4B2042C08D82146154B03EB52
S315080043D044139B68002BEAD10123E9E700240EE089
S315080043E001231D402046FFF7C3FF0F4B720103EB65
S315080043F046110431985802F0E3FE0134E4B2032C66
S315080044000AD82646084B03EB44139B68012BE8D0D1
S31508004410112BE5D00023E4E7284602B070BD00BFA3
S31508004420001002402CCF0008ACCE000808B559B1E0
S315080044300B4B4FEA401C03EB4010027F818853F870
S315080044400C0002F09CFF08BD054B4FEA401C03EB2D
S315080044504010027E818853F80C0002F090FFF2E7C4
S31508004460ACCE000838B504460D4B420103EB4015A7
S31508004470A988985802F07CFFEB69012B07D0084BF6
S3150800448003EB44139B69012B05D0002038BD012896
S31508004490F5D10120FAE708B10020F7E70120F5E792
S315080044A02CCF000808B5044B420103EB4010818865
S315080044B0985802F069FF08BDACCE00080120704785
S315080044C00246002008B10020704700EB800304492B
S315080044D051F823309342F7D0431CD8B2F2E700BF15
S315080044E0CCCF000808B5044805F0A8FC034B1860B3
S315080044F0003818BF012008BD04D00008600200205B
S3150800450038B504460378244D03EB830305EB830390
S315080045104FF0FF31586805F083FD237803EB8303DA
S3150800452005EB8303D96841F002011C4B186805F0B6
S31508004530D4FC237803EB8300A389A268616855F845
S31508004540200004F0F1F800280CBF0125002511D041
S315080045500020237810F0020F05F0010518BF00258A
S3150800456003EB83030C4A02EB8303586805F087FDC7
S31508004570284638BD237803EB8303074A02EB8303F7
S31508004580D9684FF0FF33002241F002010348006862
S3150800459005F0C3FCDDE700BFCCCF000860020020B1
S315080045A008B5FFF78DFF00EB8000044B03EB800393
S315080045B0D968034B186805F063FC08BDCCCF000822
S315080045C06002002008B5FFF77BFF00EB8000044B74
S315080045D003EB8003D968034B186805F051FC08BD46
S315080045E0CCCF00086002002008B5026E826DD26B3F
S315080045F0436DDB6BFFF764FF0221024B186805F079
S315080046003FFC08BD6002002007EE900AF8EEE77A44
S315080046109FED097A87EE870ADFED087A60EE277A3A
S315080046209FED077A77EE877A20EE270ADFED057A7F
S3150800463030EE670A704700BFECB9FE45DB8A1F41BA
S315080046406DE76B4342E0754310B52DED028B84B0E0
S3150800465000238DF80F300A2005F074FB012483E04F
S315080046609DF80F3013F0010F26D013F0800F05D1F7
S3150800467013F0400F05D04D4B019322E04C4B0193AC
S315080046801FE013F0200F02D0484B019319E013F0F6
S31508004690100F02D0454B019313E013F0080F02D018
S315080046A0424B01930DE013F0040F02D03F4B0193E8
S315080046B007E03E4B019304E013F0020F06D03B4B94
S315080046C0019300238DF80F3001245CE0374B0193EA
S315080046D0F7E79DF80F3013F0010F26D013F0800F7F
S315080046E005D113F0400F05D0304B029322E0304B32
S315080046F002931FE013F0200F02D02C4B029319E00F
S3150800470013F0100F02D0294B029313E013F0080F91
S3150800471002D0264B02930DE013F0040F02D0234B70
S31508004720029307E0214B029304E013F0020F39D0FD
S315080047301E4B029300238DF80F300124DDED018A0C
S31508004740B0EE680A0820FFF783F99DED028AB0EEFD
S31508004750480A0920FFF77CF938EEC80A0A20FFF74D
S3150800476077F9642005F0EEFA03AA0DF10F0100208F
S31508004770FFF78AFA04403FF473AFBDF80C00FFF761
S3150800478043FF8DED010A03AA0DF10F010120FFF782
S315080047907BFA04409DD0BDF80C00FFF735FF8DED80
S315080047A0020ACBE7014B0293C4E700BF7B9488C398
S315080047B00040834508B5054A0021054805F055FA25
S315080047C0044B1860003818BF012008BD30D0000817
S315080047D0494600086402002008B504F0F7FCB0FA60
S315080047E080F0400908BD70B505460E4605F0B2F9D9
S315080047F0044610F4807F04D10120E4B2FF2C0ED0C9
S3150800480070BD04F001FB0443A4B23146284605F006
S31508004810A1F9204380B2B0FA80F04009EDE7002004
S31508004820EEE7000010B502F067FBB0FA80F4640901
S31508004830024B186805F023FC204610BD68020020CC
S3150800484008B54FF0FF31054B186805F0E9FB02F093
S315080048503BFBB0FA80F0400908BD00BF68020020A3
S3150800486010B50B4805F093FB0A4B1860041E18BFD9
S315080048700124FFF7E5FF0440002004F061FE00284C
S3150800488014BF002404F00104FFF7CCFF204010BD3C
S3150800489060D0000868020020014A024B9A607047FF
S315080048A00028000800ED00E02DE9F04188B000245A
S315080048B003940494059406940794364BDA6C42F0F4
S315080048C00402DA64DA6C02F004020092009ADA6CE6
S315080048D042F00102DA64DA6C02F001020192019AEE
S315080048E0DA6C42F00202DA64DB6C03F0020302932C
S315080048F0029B294F22464FF48041384602F03FFD7D
S3150800490022464FF480714FF0904002F038FD234D57
S3150800491022466021284602F032FD4FF48043039375
S31508004920012604960594069403A9384602F048FC25
S315080049304FF40048CDF80C800494059403A9384632
S3150800494002F03EFC4FF48073039304960594069494
S3150800495003A94FF0904002F033FCCDF80C80049484
S31508004960059403A94FF0904002F02AFC982303937C
S315080049700494059403A9284602F022FC60230393B5
S3150800498004960594069403A9284602F019FC08B073
S31508004990BDE8F08100100240000800480004004805
S315080049A000B583B0164B9A6C42F001029A649A6C71
S315080049B002F001020092009A9A6C42F002029A648E
S315080049C09B6C03F002030193019B002205210C2036
S315080049D001F0CCFE0C2001F0D9FE002205210D20A5
S315080049E001F0C4FE0D2001F0D1FE002205213A2077
S315080049F001F0BCFE3A2001F0C9FE03B05DF804FBE5
S31508004A000010024008B5FEF7D5FC024B186805F001
S31508004A108AF9FEE76C02002072B6FEE700B587B099
S31508004A2000230093019302930393049305932F485D
S31508004A302F4A026043608360C36001220261082135
S31508004A404161037642760421C16180F82030836291
S31508004A50C36280F83020436380F838201C21C16384
S31508004A60802101644364826400F080FC002832D10E
S31508004A70204B009306230193072302937F23039376
S31508004A8004230493002305936946184800F0CEFED4
S31508004A9018BB194B00930C2301936946134800F081
S31508004AA0C5FEE0B9154B00931223019369460F48DA
S31508004AB000F0BCFEA8B9124B00931823019369466F
S31508004AC00A4800F0B3FE70B97F21084801F0E4F9FE
S31508004AD007B05DF804FBFFF79FFFFFF79DFFFFF7A1
S31508004AE09BFFFFF799FFFFF797FF00BF70040020B1
S31508004AF00000045040002019000021438000501D8A
S31508004B000080F03E08B50D480D4B03602023436036
S31508004B1000238360C3604FF4402202614FF4A00271
S31508004B2042610376437683760122C276037743771A
S31508004B3001F003FA00B908BDFFF76EFF0004002074
S31508004B400064004000B58BB02422002101A807F0BC
S31508004B50BAFE1048104B036001F0ABFE98B900226C
S31508004B600192029203920492059201A9094801F062
S31508004B70FBFE50B9002201A9064801F090FF30B9A2
S31508004B800BB05DF804FBFFF747FFFFF745FFFFF79C
S31508004B9043FF00BFC80300200074004008B5104852
S31508004BA0104B03604FF482734360002383604FF415
S31508004BB0E062C2600361012242614FF400728261C1
S31508004BC03022C2610362436283620722C2620363C0
S31508004BD0436303F039FD00B908BDFFF71DFF00BFA9
S31508004BE0000300200030014008B51148114B03604E
S31508004BF0114B4360002383600122C2600361436155
S31508004C008361C361036202F0C8FB50B900210848FA
S31508004C1002F021FC38B90021054802F04AFC20B907
S31508004C2008BDFFF7F9FEFFF7F7FEFFF7F5FE00BF31
S31508004C307403002000540040EC9C901008B5084806
S31508004C40084B03600623436040F6FF73C360962350
S31508004C50836002F05AFC00B908BDFFF7DDFE00BF0D
S31508004C60640300200030004008B50848084B03607C
S31508004C70002303714371436183610123036201F0D9
S31508004C80A1FD00B908BDFFF7C7FE00BFDC03002081
S31508004C900030024000B597B04422002105A807F06D
S31508004CA012FE0023009301930293039304934FF497
S31508004CB0007002F06DFC30BB092305934FF4A02366
S31508004CC0069301230A9302230F93032210920422C8
S31508004CD0119210221292072213921493159305A883
S31508004CE002F040FD88B90F230093032301930023A4
S31508004CF00293039304930421684603F069F830B9D4
S31508004D0017B05DF804FBFFF787FEFFF785FEFFF790
S31508004D1083FE000008B5FFF7BFFD00F0C3FAFFF7F2
S31508004D20B9FFFFF7C1FDFFF73BFEFFF777FEFFF779
S31508004D30E9FEFFF707FFFFF731FFFFF755FFFFF71C
S31508004D407DFFFFF791FF04F04DFF054A0021054856
S31508004D5004F08BFF044B186004F056FFFEE700BF13
S31508004D6078D00008054A00086C02002000B583B018
S31508004D700D4B1A6E42F001021A661A6E02F0010213
S31508004D800092009A9A6D42F080529A659B6D03F0E4
S31508004D9080530193019B00220F216FF0010001F05F
S31508004DA0E5FC03B05DF804FB0010024070B59EB048
S31508004DB00446002119911A911B911C911D915422A8
S31508004DC004A807F080FD2268334B9A4201D01EB032
S31508004DD070BD4FF4804304934FF04053169304A8D4
S31508004DE003F070F9002850D12C4BDA6C42F40052CB
S31508004DF0DA64DA6C02F400520192019ADA6C42F033
S31508004E000102DA64DA6C02F001020292029ADA6CA2
S31508004E1042F00202DA64DB6C03F002030393039B9D
S31508004E20062319930B261A9600251B9519A94FF0E8
S31508004E30904002F0C5F9032319931A961B9519A9F0
S31508004E40174802F0BDF91748174B0360456085609F
S31508004E50C560802303614FF4807343614FF4806318
S31508004E6083612023C3614FF40053036201F0BCFE43
S31508004E7070B90C4BE3649C6200220521122001F0F4
S31508004E8075FC122001F082FCA1E7FFF7C5FDABE730
S31508004E90FFF7C2FDEDE700BF000004500010024016
S31508004EA000040048280400203004024000B589B0F8
S31508004EB00023039304930593069307930268244BF0
S31508004EC09A4202D009B05DF804FB03F5D6339A6D11
S31508004ED042F000729A659A6D02F000720192019A88
S31508004EE0DA6C42F00102DA64DB6C03F00103029328
S31508004EF0029B4FF4C05303930223049303230693A0
S31508004F000923079303A94FF0904002F059F90022AC
S31508004F100521132001F02AFC132001F037FC00229A
S31508004F200521142001F022FC142001F02FFC002298
S31508004F300521152001F01AFC152001F027FC002296
S31508004F400521162001F012FC162001F01FFCB9E716
S31508004F50006400400268094B9A4200D0704782B04C
S31508004F60A3F500539A6C42F480529A649B6C03F43E
S31508004F7080530193019B02B0704700BF0030024086
S31508004F8000B589B00023039304930593069307930A
S31508004F900268124B9A4202D009B05DF804FB03F589
S31508004FA0CE339A6D42F000529A659A6D02F000521D
S31508004FB00192019ADA6C42F00102DA64DB6C03F0C2
S31508004FC001030293029B102303930323049303A96B
S31508004FD04FF0904002F0F4F8DEE700BF007400409E
S31508004FE010B59CB0044600211791189119911A9191
S31508004FF01B91542202A807F066FC2268184B9A42B5
S3150800500001D01CB010BD4023029302A803F05AF841
S3150800501018BB144CE36C43F00103E364E36C03F040
S3150800502001030093009B4FF4C06317931223189350
S315080050300023199303231A9304231B9317A94FF0EC
S31508005040904002F0BDF8A36D43F40013A365A36D69
S3150800505003F400130193019BD3E7FFF7DDFCD8E7C0
S31508005060005400400010024010B588B00023039396
S31508005070049305930693079302682F4B9A4201D02F
S3150800508008B010BD044603F560431A6E42F4805218
S315080050901A661A6E02F480520192019ADA6C42F08C
S315080050A00102DA64DB6C03F001030293029BE0233E
S315080050B0039302230493032306930523079303A963
S315080050C04FF0904002F07CF81C481D4B036001230A
S315080050D0436000238360C360802202614361836169
S315080050E0C361036201F080FD00BB144BA3659C629B
S315080050F01448154B03600123436010238360002383
S31508005100C3608022026143618361C361036201F067
S315080051106BFD70B90B4B63659C6200220521232049
S3150800512001F024FB232001F031FBA9E7FFF774FC0B
S31508005130DBE7FFF771FCEDE700300140B80200201D
S315080051401C0002407002002030000240FEE7FEE725
S31508005150FEE7FEE7FEE7704708B500F0B3F806F08D
S31508005160DDFC012800D108BD07F07CF9FBE700004B
S3150800517008B5024801F01FFE08BD00BFB8020020AE
S3150800518008B5024801F017FE08BD00BF70020020EE
S3150800519008B5024800F0DEF908BD00BF700400201B
S315080051A008B5024801F057F908BD00BF0004002001
S315080051B008B5024801F04FF908BD00BF00040020F9
S315080051C008B5024801F047F908BD00BF00040020F1
S315080051D008B5024801F03FF908BD00BF00040020E9
S315080051E008B5024803F02EFC08BD00BF00030020E6
S315080051F008B5024801F0DFFD08BD00BF28040020FD
S315080052000E4AD2F8883043F47003C2F888300C4B43
S315080052101A6842F001021A60002199601A6822F0A1
S31508005220A85222F410221A604FF48052DA601A68E3
S3150800523022F480221A609961704700BF00ED00E0F1
S315080052400010024008B50B460146184607F0C0FB99
S3150800525008BD0000104B1B780BB90120704710B52C
S3150800526004464FF47A70B0FBF3F30C4A1068B0FBAF
S31508005270F3F001F093FA68B90F2C01D901200AE07E
S31508005280002221464FF0FF3001F070FA044B1C60F3
S31508005290002000E0012010BD9800002094000020A6
S315080052A09C00002010B5032001F04EFA0F20FFF7EE
S315080052B0D1FF10B10124204610BD0446FFF756FD64
S315080052C0F9E70000034B1B78034A11680B44136087
S315080052D0704700BF98000020D4040020014B1868CE
S315080052E0704700BFD404002038B50446FFF7F6FF20
S315080052F00546B4F1FF3F02D0044B1B781C44FFF768
S31508005300EDFF401BA042FAD338BD00BF980000202D
S3150800531010B430300B0A9B0003F00C03C45801F09C
S315080053201F014FF01F0C0CFA01FC24EA0C0CC2F307
S3150800533084628A404CEA0202C2505DF8044B704708
S3150800534010B414304B0E9B0003F00403C458C1F389
S3150800535004514FF0070C0CFA01FC24EA0C0C8A40A5
S315080053604CEA0202C2505DF8044B704730B583B070
S3150800537000230193002800F0DA800446436D13B336
S3150800538023689A6812F0005F05D09A6822F02042D6
S3150800539022F03F029A602268936813F0805F1FD15B
S315080053A0936823F0104323F03F0343F08053936040
S315080053B0604B1B689B09604AA2FB03239B090133C8
S315080053C05B00019309E0FFF7F1FC0023A36584F86D
S315080053D05030D5E7019B013B0193019B002BF9D186
S315080053E02268936813F0805F78D1636D43F01003E9
S315080053F06365A36D43F00103A3650120936813F069
S31508005400040300D00123616D11F0100F40F088806D
S31508005410002B40F08580636D23F4817343F002030B
S315080054206365936813F0010F0BD1444B9B6813F027
S31508005430010F06D1636842498A6822F47C12134335
S315080054408B60627E636B43EA4233E2681343A26869
S31508005450134394F8202043EA0243012A40D0A26A63
S3150800546022B102F47072E16A0A4313432168CD68D7
S31508005470344A2A401A43CA6021688B6813F0040329
S3150800548000D001238A6812F0080200D00122B3B9BD
S31508005490AAB9237E94F83020520042EA8332CB68B8
S315080054A023F4804323F002031343CB6094F8383087
S315080054B0012B1AD02268136923F0010313612369AB
S315080054C0012B24D02268136B23F00F031363636D3B
S315080054D023F0030343F00103636526E000208DE70C
S315080054E0626A013A43EA4243B9E721680B6923F441
S315080054F0FF6323F00403E26B256C2A43656C2A4399
S31508005500A56C2A43134343F001030B61D7E72168CF
S315080055100B6B23F00F03E269013A13430B63D6E7DB
S31508005520636D43F010036365012003B030BD0120AD
S31508005530FBE700BF94000020632D3E0500000450E1
S315080055400003045007C0F0FF08B5806AFEF748FD5F
S3150800555008BD704770B5044603681E685D6816F096
S31508005560020F10D015F0020F0DD0436D13F0100F77
S3150800557003D1436D43F400634365204600F0DCFC29
S31508005580236802221A6016F0040F02D015F0040FE1
S3150800559005D116F0080F3AD015F0080F37D0636D0D
S315080055A013F0100F03D1636D43F40073636523682A
S315080055B0DA6812F4406F24D1DA6812F4005F20D159
S315080055C01A6812F0080F1CD09A6812F0040F10D14E
S315080055D05A6822F00C025A60636D23F4807363657F
S315080055E0636D13F4805F0CD1636D43F0010363654B
S315080055F007E0636D43F010036365A36D43F0010391
S31508005600A3652046FEF7E2FC23680C221A6016F012
S31508005610200F02D015F0200F05D116F0400F4CD000
S3150800562015F0400F49D0636D13F0100F03D1636D69
S3150800563043F4005363652368DA6C12F0C00F2AD16D
S315080056400121DA6812F4406F27D10120DA6871B3B4
S3150800565012F0007F03D050B312F4005F27D1196807
S3150800566011F0400F23D012F4001F20D19A6812F0CF
S31508005670080F14D15A6822F060025A60636D23F449
S3150800568080536365636D13F4807F10D1636D43F0B7
S31508005690010363650BE00021D3E70020D6E7636DBD
S315080056A043F010036365A36D43F00103A365204629
S315080056B000F03EFC236860221A6016F0800F02D0C4
S315080056C015F0800F2DD116F4807F02D015F4807F57
S315080056D032D116F4007F02D015F4007F38D116F0C7
S315080056E0100F17D015F0100F14D0636B23B1236871
S315080056F0DB6813F0010F0AD0636D43F480636365BA
S31508005700A36D43F00203A3652046FEF773FC2368E6
S3150800571010221A6016F4806F02D015F4806F23D118
S3150800572070BD636D43F4803363652046FFF711FF50
S31508005730236880221A60C6E7636D43F40033636505
S31508005740204600F0F7FB23684FF480721A60C0E722
S31508005750636D43F480236365204600F0ECFB236801
S315080057604FF400721A60BAE7636D43F480436365C9
S31508005770A36D43F00803A36523684FF480621A609B
S31508005780204600F0D6FBCBE708B50346806A426D93
S3150800579012F0500F30D1436D43F40073436503682C
S315080057A01A6812F0080F14D0DA6812F4406F20D184
S315080057B0DB6813F4005F1CD1436D23F480734365E3
S315080057C0436D13F4805F14D1436D43F001034365C1
S315080057D00FE0DB6813F0020F0BD1436D23F48073DF
S315080057E04365436D13F4805F03D1436D43F00103B2
S315080057F04365FEF7EBFB08BD426D12F0100F04D1AE
S31508005800C26C526B18469047F5E7FEF7F3FBF2E7D2
S3150800581008B5806A436D43F040034365836D43F0E2
S3150800582004038365FEF7E6FB08BD0000F0B583B008
S315080058300023019390F85030012B00F00A820446A9
S315080058400D46012380F8503003689B6813F0040F57
S3150800585009D0436D43F0200343650120002384F8F3
S31508005860503003B0F0BD4B68052B08D8023B032B1C
S3150800587056D8DFE803F0024B4E510C234B602A68DA
S3150800588069682068FFF744FD2068836813F00403FD
S3150800589000D00123826812F0080200D001220BB959
S315080058A0002A40D02268936813F0010F17D12B689D
S315080058B0E868D2F8B010C3F3120621EA060100F030
S315080058C0180CAA4820FA0CF00340C3F312030B4342
S315080058D0C2F8B030EA68A64B9A4200F0A9802B6855
S315080058E0A44A134200F0B181A34A926802F0E0701C
S315080058F0A2498B4200F05B81A1498B4200F07E8170
S31508005900A0498B4200F08E810020A7E712234B6046
S31508005910B5E718234B60B2E74FF480734B60AEE7E8
S3150800592006234B60ABE7AA682968FFF709FD696992
S315080059302268D368C3F3C1035B0099402869042829
S315080059400ED02E68603252F820708F4B3B4006F01E
S31508005950F84631430B4343F0004342F82030A1E7B1
S31508005960136E116EC1F384612B68C3F3120080BBFA
S31508005970C3F38463994234D021684B6E4A6EC2F3EE
S3150800598084622B68C3F3120080BBC3F384639A4214
S3150800599034D021688B6E8A6EC2F384622B68C3F397
S315080059A0120080BBC3F384639A4234D02168CB6E5D
S315080059B0CA6EC2F384622B68C3F3120080BBC3F3BA
S315080059C084639A427FF46EAFCB6E23F00043CB66B6
S315080059D068E793FAA3F313B1B3FA83F3CAE720236C
S315080059E0C8E7136E23F000431366C5E793FAA3F3DB
S315080059F013B1B3FA83F3CAE72023C8E74B6E23F043
S31508005A0000434B66C5E793FAA3F313B1B3FA83F3DE
S31508005A10CAE72023C8E78B6E23F000438B66C5E7E9
S31508005A2093FAA3F313B1B3FA83F3CAE72023C8E7BB
S31508005A3020682B68C3F312063EBB9A0E013202F0A9
S31508005A401F02092A8CBF00220122002A55D05EBBFC
S31508005A50990E0131890601F0F8418EBB4FEA936C25
S31508005A600CF1010C0CF01F0C012202FA0CF2114386
S31508005A70AEBB9B0E013303F01F0303EB43031B0569
S31508005A801943AA68FFF75CFC29E793FAA3F24AB11F
S31508005A90B2FA82F2013202F01F02092A8CBF0022F2
S31508005AA00122D2E72022F5E793FAA3F131B1B1FA40
S31508005AB081F10131890601F0F841CEE72021F8E7A6
S31508005AC093FAA3F24AB1B2FA82F2013202F01F0245
S31508005AD04FF0010C0CFA02F2C9E72022F5E793FA17
S31508005AE0A3F343B1B3FA83F3013303F01F0303EBC4
S31508005AF043031B05C4E72023F6E7E6B9990E0131EF
S31508005B00890601F0F84116BB4FEA936C0CF1010CBB
S31508005B100CF01F0C012202FA0CF21143B6BB9B0EC5
S31508005B20013303F01F0303EB43031E3B1B0543F03E
S31508005B3000731943A5E793FAA3F131B1B1FA81F1DC
S31508005B400131890601F0F841DDE72021F8E793FAEB
S31508005B50A3F24AB1B2FA82F2013202F01F024FF002
S31508005B60010C0CFA02F2D8E72022F5E7FFFF07003E
S31508005B7000007F400000088000030450000052C760
S31508005B80000084CB0100008000F0FF0393FAA3F322
S31508005B905BB1B3FA83F3013303F01F0303EB43034B
S31508005BA01E3B1B0543F00073C3E72023F3E712F4FB
S31508005BB0000F7FF4A1AE2268274B9A4201D000203D
S31508005BC04CE640F4000325498A6822F0E072134344
S31508005BD08B60234B1B689B09224AA2FB03239B0964
S31508005BE0013303EB43039B00019302E0019B013B56
S31508005BF00193019B002BF9D100202FE612F0807F3C
S31508005C007FF47EAE2268144B9A4201D0002025E626
S31508005C1040F0807311498A6822F0E07213438B6062
S31508005C2000201BE612F4800F11D122680A4B9A4213
S31508005C3001D0002012E640F4800308498A6822F061
S31508005C40E07213438B60002008E6002006E6002079
S31508005C5004E6022005E600BF0000045000030450D5
S31508005C6094000020632D3E0530B583B000230193D0
S31508005C7003689A6812F0010F58D1044699682D4AAC
S31508005C80114219D19A6822F0004222F03F0242F0EE
S31508005C9001029A60284B9B6813F4000F1CD0274B0F
S31508005CA01B689B09264AA2FB03239B09013303EBC6
S31508005CB043039B0001930CE0436D43F010034365D7
S31508005CC0836D43F001038365012030E0019B013BAE
S31508005CD00193019B002BF9D1FFF700FB05462368CA
S31508005CE01A6812F0010F1FD19A6812F0010F07D136
S31508005CF09A6822F0004222F03F0242F001029A60BE
S31508005D00FFF7ECFA431B022BE9D923681B6813F04B
S31508005D10010FE4D1636D43F010036365A36D43F08F
S31508005D200103A365012002E0002000E0002003B083
S31508005D3030BD00BF3F0000800003045094000020DF
S31508005D40632D3E0570B504460068806810F0040FA0
S31508005D504ED10E46154694F85030012B4AD00123F1
S31508005D6084F850302046FFF77FFF00283CD1636D4A
S31508005D7023F4706323F0010343F480736365636D52
S31508005D8013F4805F2DD0A36D23F00603A365E36C9F
S31508005D90194ADA62E36C194A1A63E36C184A5A63B9
S31508005DA023681C221A60002384F85030226853683E
S31508005DB043F0100353602268D36843F00103D360AD
S31508005DC021682B4632464031E06C00F091FF22688C
S31508005DD0936823F0004323F03F0343F004039360E2
S31508005DE007E00023A365D2E7002384F8503000E0DB
S31508005DF0022070BD0220FCE78957000849550008B3
S31508005E001158000838B504460268936813F002036F
S31508005E1000D00123916811F0010F39D0002B39D138
S31508005E20936803F00D03012B09D0636D43F010034B
S31508005E306365A36D43F00103A365012029E0936818
S31508005E4023F0004323F03F0343F0020393602368E3
S31508005E5003221A60FFF742FA054623689B6813F087
S31508005E60010F13D0FFF73AFA401B0228F5D9236829
S31508005E709B6813F0010FF0D0636D43F01003636560
S31508005E80A36D43F00103A365012002E0002000E0B2
S31508005E90002038BD0020FCE730B583B0002301930D
S31508005EA090F85030012B41D004460D46012380F866
S31508005EB05030FFF7A7FF80BB636D23F4885323F0A8
S31508005EC0020343F0020363652268936823F04043A4
S31508005ED023F03F0305F080452B4343F000439360CE
S31508005EE023689B68002B06DB636D23F0030343F0EE
S31508005EF00103636515E0019B01330193019BB3F52B
S31508005F00912FEDD3636D23F0120343F010036365FD
S31508005F10002384F85030012006E0636D43F0100337
S31508005F206365002384F8503003B030BD0220FBE7D8
S31508005F3070477047704770477047002800F0A18087
S31508005F4038B5044690F82030D3B12268136843F078
S31508005F5001031360FFF7C2F9054623685A6812F071
S31508005F60010F10D1FFF7BAF9401B0A28F5D9636A61
S31508005F7043F400336362052384F82030012038BDDA
S31508005F80FEF794FFE1E71A6822F002021A60FFF7AB
S31508005F90A5F9054623685A6812F0020F0DD0FFF7D7
S31508005FA09DF9401B0A28F5D9636A43F400336362F6
S31508005FB0052384F820300120E1E7227E012A3DD01E
S31508005FC01A6822F080021A60637E012B3BD0226891
S31508005FD0136823F040031360A37E012B39D022688F
S31508005FE0136823F020031360E37E012B37D0226861
S31508005FF0136843F010031360237F012B35D0226802
S31508006000136823F008031360637F012B33D02268DB
S31508006010136823F004031360A368E2681343226934
S315080060201343626913436268013A21681343CB61DB
S3150800603000206062012384F82030A0E71A6842F045
S3150800604080021A60C0E72268136843F040031360B1
S31508006050C2E72268136843F020031360C4E7226886
S31508006060136823F010031360C6E72268136843F029
S3150800607008031360C8E72268136843F00403136033
S31508006080CAE701207047026890F82030013BDBB26E
S31508006090012B05D9436A43F48023436201207047E4
S315080060A030B4D2F8003243F00103C2F800324B692B
S315080060B003F01F03012000FA03F3D2F81C026FEA6B
S315080060C0030C20EA0300C2F81C02C869B0B9D2F86A
S315080060D00C020CEA0000C2F80C028C884869CD68EC
S315080060E044EA0544483042F830400C8848698D68CF
S315080060F044EA0544483002EBC0004460C8690128F8
S315080061001BD0886980BBD2F804020CEA0000C2F8EA
S315080061100402086970BBD2F814020CEA0000C2F83F
S315080061201402096A01292BD0D2F8003223F00103A0
S31508006130C2F80032002030BC7047D2F80C0218436F
S31508006140C2F80C028C8848690D6844EA0544483050
S3150800615042F830408C8948698D6844EA05444830DD
S3150800616002EBC0004460CCE7D2F804021843C2F838
S315080061700402CEE7D2F814021843C2F81402D0E794
S31508006180D2F81C120B43C2F81C32CDE770B5044690
S3150800619090F82050EDB2012D06D0436A43F400234F
S315080061A043620125284670BD022380F82030026824
S315080061B0136823F001031360FFF790F80646236877
S315080061C05B6813F0010F0CD0FFF788F8831B0A2BC6
S315080061D0F5D9636A43F400336362052384F82030F3
S315080061E0E0E700256562DDE730B590F820C0046871
S315080061F0A4680CF1FF3C5FFA8CFCBCF1010F62D875
S3150800620014F0E05F59D0C4F3016C012404FA0CF4CD
S315080062101C608B68002B3DD10D68CB68046843EA87
S3150800622045550CF118031B01E55003680C690CF180
S31508006230180E03EB0E135C600B7D012B35D0D1795C
S3150800624093791B0443EA0163517943EA01231479DC
S315080062500168234301EB0C11C1F88C31D17893788E
S315080062601B0443EA0163517843EA01231178026863
S315080062700B4302EB0C12C2F8883102680CF1180CB9
S315080062804FEA0C1C52F80C3043F0010342F80C306C
S3150800629000201DE04C6843EAC403CC6823430CF194
S315080062A01804240105682B51BFE7036803EB0E1396
S315080062B0596841F480715960C1E7436A43F4001391
S315080062C04362012004E0436A43F4802343620120C9
S315080062D030BD90F820C00CF1FF3C5FFA8CFCBCF195
S315080062E0010F00F2958030B451B90468E46814F0DF
S315080062F0030F10D1436A43F400134362012077E089
S315080063000468246914F0030F05D1436A43F40013A3
S31508006310436201206CE001F11B04240105682C5935
S3150800632004F004049460002C64D101F11B042401D8
S3150800633005682C59640D1460046801F11B0C4FEABA
S315080063400C1C54F80C4004F00204D460046864443D
S31508006350646804F00F041461046864446468C4F350
S3150800636007249461046864446468240C54610268D0
S3150800637002EB0112D2F8B8211A70026802EB011278
S31508006380D2F8B821C2F307225A70026802EB01124A
S31508006390D2F8B821C2F307429A70026802EB0112DA
S315080063A0D2F8B821120EDA70026802EB0112D2F89E
S315080063B0BC211A71026802EB0112D2F8BC21C2F3A1
S315080063C007225A71026802EB0112D2F8BC21C2F305
S315080063D007429A71026802EB0112D2F8BC21120E2A
S315080063E0DA7179B90268D36843F02003D3600020D4
S315080063F030BC704701F11B04240105682C59E408D8
S31508006400546099E70268136943F020031361EEE7C5
S31508006410436A43F4802343620120704790F8203092
S31508006420013BDBB2012B05D9436A43F4802343625F
S3150800643001207047026853690B4353610020704777
S315080064407047704770477047704770477047704786
S315080064507047704770472DE9F84F054603685C6931
S31508006460D3F804809F68D3F80CB0D3F810A0D3F8FB
S31508006470189014F001063BD017F0010616D0012239
S315080064809A6017F0020F08D117F0040F0CD117F015
S31508006490080606D04FF4805608E0FFF7D1FF00261D
S315080064A004E0FFF7D0FF01E04FF4006617F4807FA1
S315080064B00DD02B684FF480729A6017F4007F40F075
S315080064C0868017F4806F00F0868046F4005617F42D
S315080064D0803F0DD02B684FF480329A6017F4003F46
S315080064E040F0838017F4802F00F0838046F400463E
S315080064F014F0080F07D01BF0100F04D046F40076EE
S315080065002B681022DA6014F0040F02D01BF0080F73
S3150800651079D114F0020F04D02B68DB6813F0030F4F
S3150800652078D114F0400F07D01AF0100F04D046F4B3
S3150800653080662B6810221A6114F0200F02D01AF018
S31508006540080F6BD114F0100F04D02B681B6913F0D9
S31508006550030F6AD114F4003F02D018F0100F68D167
S3150800656014F4803F02D018F0080F69D114F4004FD4
S315080065707AD018F0040F74D014F4807F04D019F080
S31508006580010F01D046F0010614F4007F04D019F07B
S31508006590020F01D046F0020614F4806F04D019F0F9
S315080065A0040F01D046F0040614F4006F59D019F010
S315080065B0700956D0B9F1400F65D058D8B9F1200FF7
S315080065C05ED0B9F1300F42D146F0200644E02846A5
S315080065D0FFF737FF7BE717F4006F02D046F48046D3
S315080065E075E72846FFF730FF71E72846FFF72AFFC9
S315080065F07EE717F4002F02D046F4803678E728465F
S31508006600FFF723FF74E72B680822DA602846FFF7AE
S315080066101DFF7EE72846FDF777FE82E72B680822EE
S315080066201A612846FFF714FF8CE72846FFF70FFF85
S3150800663090E72B6810225A602846FFF70AFF8FE773
S315080066402B6808225A602846FFF704FF8EE7B9F13F
S31508006650100F01D146F008062A68936923F07003E3
S3150800666093612B6804225A609EB9BDE8F88FB9F188
S31508006670500F0BD0B9F1600FEED146F48076EBE7F8
S3150800668046F01006E8E746F04006E5E746F08006DD
S31508006690E2E76B6A33436B622846FDF757FEE4E789
S315080066A0002807DB00F01F02400901239340024A35
S315080066B042F82030704700BF00E100E0002808DB00
S315080066C00901C9B200F1604000F5614080F8001385
S315080066D0704700F00F000901C9B2014B1954704701
S315080066E014ED00E000B500F00700C0F1070CBCF19E
S315080066F0040F28BF4FF0040C031D062B0FD9C31E29
S315080067004FF0FF3E0EFA0CF021EA000199400EFA0E
S3150800671003FE22EA0E0241EA02005DF804FB0023AA
S31508006720EEE70000BFF34F8F0549CA6802F4E0623E
S31508006730044B1343CB60BFF34F8F00BFFDE700BF89
S3150800674000ED00E00400FA05074AD36823F4E06385
S315080067501B041B0C000200F4E060034343F0BF6314
S3150800676043F40033D360704700ED00E010B50446EB
S31508006770054BD868C0F30220FFF7B4FF0146204650
S31508006780FFF79CFF10BD00BF00ED00E008B5FFF75E
S3150800679087FF08BD08B5FFF7C5FF00000138B0F14F
S315080067A0807F0BD24FF0E0235861054AF02182F82A
S315080067B023100020986107221A617047012070474C
S315080067C000ED00E0002838D010B50446437F1BB31F
S315080067D00223637723791BBB2368194A5A61226807
S315080067E0936823F018039360637913BB23684FF00B
S315080067F0FF321A612268936823F0600361690B43CC
S3150800680093602268936823F08003A1690B43936021
S3150800681001236377002010BD0377FEF79BFBD7E7BC
S31508006820E268A168204600F00DF80028DCD00120B7
S31508006830F1E7236822691A61DCE70120704700BF87
S31508006840B71DC10410B41F231C46013B34B103F025
S315080068501F0C21FA0CFC1CF0010FF5D0182A22D8BF
S31508006860DFE802F00F212121212121211D212121EB
S315080068702121212119212121212121210D00062B48
S3150800688015D80368596101688B6823F01803134308
S315080068908B60002008E0072BF3D9012004E00F2BBA
S315080068A0EFD9012000E001205DF8044B7047012074
S315080068B0FAE770B110B50446037933B102232371A0
S315080068C0002020610123237110BD4371FEF758FB98
S315080068D0F4E7012070474279012A2CD010B4034608
S315080068E001224271022018711C68206801F0100C00
S315080068F002FA0CF20243226089B919680A6802F0A2
S315080069003C02042A06D001221A71002058715DF84B
S31508006910044B70474A6842F001024A60F3E7196877
S315080069200A6802F47012B2F5802FECD14A6842F078
S3150800693002024A60E7E70220704710B483B00024D9
S3150800694001940068019051B901990A4408320192EC
S31508006950019A1360002003B05DF8044B7047019953
S315080069600A4414320192F3E7F8B54379012B00F093
S31508006970948004460D46164601234371022303718B
S315080069800B68042B32D02B69012B79D02068C16B98
S3150800699006F010020723934021EA03012B68AE682C
S315080069A03343EE68334393400B43C363206803685D
S315080069B04FF48041914023EA01030360206801688F
S315080069C040F6FC73934021EA03016B6893400B433E
S315080069D0036020680368C02101FA02F223EA020371
S315080069E003600123237100206071F8BDFEF776FC71
S315080069F007467EB123685B6B002B3ADAFEF76EFC1E
S31508006A00C01B0128F6D9236943F008032361032034
S31508006A102071EAE723685B6B13F4004F0BD0FEF78F
S31508006A205DFCC01B0128F5D9236943F008032361DF
S31508006A3003202071D9E70120FEF756FC2368AA69CE
S31508006A401A642068836C06F0100240F2FF31914008
S31508006A5023EA0103E96991400B4383642068C36C08
S31508006A60FF21914023EA0103296A91400B43C3643D
S31508006A7089E70120FEF738FC2368AA695A64E0E72B
S31508006A8021688A6B06F010001F23834022EA03025E
S31508006A906B69834013438B6378E70220A5E70028D8
S31508006AA000F083802DE9F04F83B0894604460379C8
S31508006AB0DBB2022B7BD04379012B7AD001214171BD
S31508006AC00068C56B02F010070723BB4005EA030BF5
S31508006AD00568B94025EA010101602068C16B6FEAC3
S31508006AE0030A21EA0303C3632368019392B9019B4E
S31508006AF008330193019B4FF400621A6022681368F9
S31508006B004FF4804808FA07F843EA08031360082593
S31508006B10102605E0019B14330193EBE72E446D081C
S31508006B209DB121688B6B1F22BA4023EA020306FA3D
S31508006B3007F213438B630120FEF7D6FB23685B6BD2
S31508006B4038EA0303EAD1761BE9E721688B6B1F2233
S31508006B50BA40D54323EA020306FA07F213438B63C6
S31508006B600120FEF7C1FB23685A6B18EA020F06D10B
S31508006B7001369A6B154006FA07F73D439D6322686E
S31508006B80136823EA08031360C9F814600123C9F8D7
S31508006B9010302268D36B0AEA030A4AEA0B03D36366
S31508006BA00020607103B0BDE8F08F01207047012016
S31508006BB0F8E70220F6E730B4446C04F01C0C012414
S31508006BC004FA0CF4056C6C60046863608368102B27
S31508006BD005D0036899600368DA6030BC70470368BB
S31508006BE09A600368D960F8E7002873D010B40346A2
S31508006BF00068394A90424AD8384A02443849A1FBC3
S31508006C000212120992005A64364A1A64022283F85A
S31508006C102520016821F4FF4121F070019A68DC689B
S31508006C2022431C6922435C6922439C692243DC692E
S31508006C3022431C6A22430A4302609A68B2F5804FCF
S31508006C401BD0196C274A91422CD0264AD2F8A81490
S31508006C50586C00F01C0C0F2000FA0CF021EA000119
S31508006C60C2F8A814D2F8A81458685C6C04F01C0C76
S31508006C7000FA0CF00143C2F8A8140020D8630122D8
S31508006C8083F8252083F824005DF8044B7047164ADC
S31508006C9002441349A1FB0212120992005A64134ACC
S31508006CA01A64B3E7D2F8A810586C00F01C0C0F2031
S31508006CB000FA0CF021EA0001C2F8A810D2F8A810D0
S31508006CC058685C6C04F01C0C00FA0CF00143C2F81E
S31508006CD0A810D2E70120704707040240F8FFFDBF5D
S31508006CE0CDCCCCCC00000240F8FBFDBF000402402E
S31508006CF038B5044690F82400012832D0012084F8DB
S31508006D00240094F82500C0B2012804D0002384F892
S31508006D102430022038BD022084F825000020E063D4
S31508006D202568286820F0010028602046FFF743FF01
S31508006D30236B5BB12268136843F00E031360226865
S31508006D40136843F0010313600020E3E72268136821
S31508006D5023F0040313602268136843F00A031360E0
S31508006D60EDE70220D6E708B590F82530DBB2022B0E
S31508006D7003D00423C363012008BD0268136823F007
S31508006D800E0313600268136823F001031360436C53
S31508006D9003F01C03016C012202FA03F34B6080F82E
S31508006DA02520002380F82430836B13B198470020F0
S31508006DB0E2E70020E0E738B5036C1968046825683F
S31508006DC0436C03F01C0304229A400A4215D015F0BE
S31508006DD0040F12D0236813F0200F03D1236823F081
S31508006DE004032360436C03F01C02016C04239340E4
S31508006DF04B60036B03B1984738BD02229A400A429A
S31508006E001CD015F0020F19D0236813F0200F06D1F5
S31508006E10236823F00A032360012380F82530436C96
S31508006E2003F01C02016C022393404B60002380F898
S31508006E302430C36A002BDFD09847DDE7082202FA20
S31508006E4003F30B42D8D015F0080FD5D0236823F0EA
S31508006E500E032360436C03F01C03016C012202FA43
S31508006E6003F34B60C26380F82520002380F82430A2
S31508006E70436B002BC0D09847BEE7000010B4064C01
S31508006E80616941F0010161610260BFF36F8F436080
S31508006E905DF8044B704700BF00200240094A536959
S31508006EA043F480235361EFF3108C72B6402351F8F4
S31508006EB0042B40F8042B013B13F0FF03F7D18CF3A6
S31508006EC01088704700200240094B5B69002B01DBE4
S31508006ED000207047064B074A9A6002F188329A608A
S31508006EE05B69002B01DB002070470120704700BF5B
S31508006EF00020024023016745034A536943F00043D3
S31508006F0053610020704700BF0020024038B5044690
S31508006F10FEF7E4F90546144B1B6913F4803F09D0C4
S31508006F20B4F1FF3FF7D0FEF7D9F9401BA042F2D3E0
S31508006F30032015E00C4B1B690C4A134009D10A4B78
S31508006F401B6913F0010F0CD0074B01221A610020B0
S31508006F5006E007494A681A434A60034A1361012052
S31508006F6038BD0020FCE700BF00200240FAC302003B
S31508006F70A00000202DE9F0411646284A1278012A79
S31508006F8049D004460D469846244B01221A704CF205
S31508006F905030FFF7BBFF074608BB204B00225A605C
S31508006FA01F4B1B6813F4806F1FD01D4A136823F408
S31508006FB080631360194B02221A77D4B1631E012B22
S31508006FC01ED900244CF25030FFF7A0FF074624B123
S31508006FD0134A536923EA0403536100F047F80F4B39
S31508006FE000221A703846BDE8F0810C4B00221A7749
S31508006FF0E3E7324643462846FFF740FF0124E1E728
S3150800700031462846FFF74AFF022C01D00024D9E76B
S315080070104FF48024D6E70227E4E700BFA00000204B
S315080070200020024010F0010F04D0054A536943F0CE
S3150800703004035361024A536943F48033536170472A
S3150800704000200240084B5A6922F47E72C00000F400
S31508007050FF6002435A615A6942F002025A615A694C
S3150800706042F480325A61704700200240164B1B7F5B
S31508007070DBB2012B01D0032B10D1144A116821F47D
S3150800708000711160116841F400611160116821F402
S3150800709000611160116841F400711160023BDBB2B6
S315080070A0012B03D9084B00221A777047074B1A6839
S315080070B042F480521A601A6822F480521A601A68DA
S315080070C042F480621A60EDE7A0000020002002402A
S315080070D0F8B5394B1B78012B6BD004460E46364B58
S315080070E001221A704CF25030FFF710FF07460028AD
S315080070F05AD1314B00225A60304B1B6813F4007F7B
S315080071002FD02E4B1B6813F4806F26D02B4A13689A
S3150800711023F480631360284B03221A772368012B14
S3150800712031D04FF0FF333360A568A368E268134493
S31508007130AB4237D961682846FFF784FF4CF25030D6
S31508007140FFF7E4FE1D4A536923F47E7323F0020316
S315080071505361074628BB0135E7E7174B01221A7723
S31508007160DCE7164B1B6813F4806F08D0134A1368C4
S3150800717023F480631360104B02221A77CEE70E4B76
S3150800718000221A77CAE76068FFF74CFF4CF25030C6
S31508007190FFF7BCFE0746094A536923F00403536107
S315080071A000E03560FFF762FF034B00221A7038468D
S315080071B0F8BD0227FBE700BFA00000200020024020
S315080071C0F0B583B0002362E085685E000324B4400E
S315080071D025EA0405CC68B4402C438460456825EA52
S315080071E00C054C68C4F300149C402C4344605FE0D3
S315080071F0DD08083550F8254003F0070C4FEA8C0CDB
S315080072004FF00F0E0EFA0CFE24EA0E0E0C6904FA65
S315080072100CF444EA0E0440F8254060E0022400E03D
S31508007220002404FA0EF42C430CF1020C4C4D45F8DC
S315080072302C404C4CA568D44325EA02064F6817F43F
S31508007240801F01D042EA0506464DAE60ED6804EAA5
S3150800725005064F6817F4001F01D042EA0506414D9E
S31508007260EE606D6804EA05064F6817F4003F01D022
S3150800727042EA05063B4D6E602D682C404E6816F4B2
S31508007280803F01D042EA0504364A146001330A6891
S3150800729032FA03F462D04FF0010C0CFA03FC1CEA34
S315080072A00202F3D04C6804F00304013C012C8BD98C
S315080072B04C6804F00304032C0CD0C4685D004FF03E
S315080072C0030C0CFA05FC24EA0C0C8C68AC4044EA66
S315080072D00C04C4604C6804F00304022C88D00468CB
S315080072E04FEA430E4FF0030C0CFA0EFC24EA0C0C82
S315080072F04C6804F0030404FA0EF444EA0C0404602F
S315080073004C6814F4403FC1D0174C256E45F0010572
S315080073102566246E04F001040194019C4FEA930C3F
S315080073200CF102050E4C54F8255003F0030E4FEAF3
S315080073308E0E0F2404FA0EF425EA0405B0F1904FD8
S315080073403FF46EAF094CA04206D004F58064A04213
S315080073503FF464AF072464E7012462E703B0F0BD95
S3150800736000000140000401400010024000040048EB
S315080073700369194201D001207047002070470AB1FD
S315080073808161704781627047436901EA030221EA15
S31508007390030141EA024181617047002859D010B5BE
S315080073A0044690F84130002B43D0242384F841301A
S315080073B02268136823F0010313606368226823F0C8
S315080073C0706313612268936823F400439360E3684B
S315080073D0012B33D0A368226843F404439360E3681F
S315080073E0022B31D02268536843F0007343F40043FC
S315080073F053602268D36823F40043D3602369626923
S315080074001343A169226843EA0123D360E369216A29
S3150800741022680B4313602268136843F00103136064
S3150800742000206064202384F84130206384F84200F9
S3150800743010BD80F84030FDF7D3FDB6E7A368226893
S3150800744043F400439360CAE723684FF400625A6026
S31508007450C8E701207047034690F84120D2B2202A97
S3150800746023D190F84020012A21D0012280F840201B
S31508007470242280F841200068026822F00102026096
S315080074801868026822F4805202601868026811437C
S31508007490016019680A6842F001020A60202283F82E
S315080074A04120002083F840007047022070470220E0
S315080074B07047034690F84120D2B2202A21D190F88D
S315080074C04020012A1FD0012280F84020242280F87B
S315080074D041200068026822F001020260186802680A
S315080074E022F4706242EA0122026019680A6842F0D0
S315080074F001020A60202283F84120002083F8400018
S315080075007047022070470220704700282FD038B5F0
S31508007510044603684CF6CC421A60036845F2555295
S315080075201A60036842685A60036882689A60FDF7C1
S31508007530D5FE05462368DA6812F0070F0BD0FDF76B
S31508007540CDFE401B3128F5D92368DB6813F0070FF9
S31508007550F0D0032005E01969E268914202D01A6169
S31508007560002038BD4AF6AA221A600020F9E7012051
S31508007570704703684AF6AA221A600020704700007E
S31508007580024B186800F4C060704700BF00700040E6
S31508007590B0F5007F0FD01F4B1B6803F4C063B3F52B
S315080075A0806F34D01B4A136823F4C06343F48063A6
S315080075B0136000207047174B1B6803F4C063B3F5CC
S315080075C0007F20D0134A136823F4C06343F4007382
S315080075D01360114B1B68322202FB03F30F4AA2FB0E
S315080075E003239B0C013300E0013B0A4A526912F45B
S315080075F0806F01D0002BF7D1064B5B6913F4806FBF
S3150800760003D10020704700207047032070470020F0
S31508007610704700BF007000409400002083DE1B43C3
S3150800762030B583B00446204B9B6D13F0805F0BD0BA
S31508007630FFF7A6FFB0F5007F17D0802C1FD82DD0F6
S31508007640702C2DD000211BE0174DAB6D43F08053F5
S31508007650AB65AB6D03F080530193019BFFF790FF79
S31508007660AB6D23F08053AB65E4E7802C03D9A02CDF
S3150800767003D9022104E0002102E0012100E00321F0
S315080076800A4A136823F007030B431360136803F0D1
S3150800769007038B4206D1002003B030BD0221EFE775
S315080076A00121EDE70120F7E7001002400020024023
S315080076B0284A9368D26802F0030213F00C030AD032
S315080076C00C2B06D0042B1FD0082B20D000200246F6
S315080076D010E0012AF6D11F4A126812F0080F0CD1E1
S315080076E01C4AD2F89420C2F303221B4951F82220DF
S315080076F043B100200C2B0DD07047164A1268C2F30E
S315080077000312F2E71046F5E714480022F2E7144898
S315080077100022EFE70F4BDB6803F00303022B16D0BA
S31508007720032B00D10E4A0B49CB68C3F3021301336E
S31508007730C868C0F3062002FB00F0B0FBF3F0CB6884
S31508007740C3F3416301335B00B0FBF3F0D4E7034AAC
S31508007750E9E700BF001002409CD000080024F400AE
S31508007760005A6202002800F01C83F0B583B0044674
S31508007770964B9D6805F00C05DE6806F0030603685F
S3150800778013F0100F5AD0E5B10C2D18D0A369002BB1
S3150800779000F0BB808D4A136843F001031360FDF7C0
S315080077A09DFD0746894B1B6813F0020F40F09A802F
S315080077B0FDF794FDC01B0228F4D90320FCE2012E34
S315080077C0E4D1824B1B6813F0020F03D0A369002B88
S315080077D000F0E982206A7D4B1B6813F0080F5BD026
S315080077E07A4B1B6803F0F00398425CD8774B1A680B
S315080077F042F008021A601A6822F0F002216A0A4367
S315080078001A605A6822F47F42E16942EA01225A6004
S31508007810002D60D0FFF74CFF6C4B9B68C3F3031336
S315080078206B4AD35C03F01F03D8406A4B18606A4B57
S315080078301868FDF70FFD002840F0BE82236813F094
S31508007840010F00F08180082D75D00C2D71D063686A
S31508007850B3F5803F00F09780B3F5A02F00F099802C
S315080078605A4B1A6822F480321A601A6822F4802267
S315080078701A606368002B00F09980FDF72FFD074614
S31508007880524B1B6813F4003F5ED1FDF727FDC01B62
S315080078906428F5D903208FE24C4BD3F894301B09A2
S315080078A003F0F003A0E7FFF7BBFE002840F07D8257
S315080078B0464B1A6842F008021A601A6822F0F0026B
S315080078C0216A0A431A605A6822F47F42E16942EA49
S315080078D001225A609EE7206AFFF7A2FE002899D087
S315080078E0012069E2394B1A6842F008021A601A68E0
S315080078F022F0F002216A0A431A605A6822F47F428B
S31508007900E16942EA01225A6098E7304A136823F08F
S3150800791001031360FDF7E2FC07462C4B1B6813F0C6
S31508007920020F8BD0FDF7DAFCC01B0228F5D903201D
S3150800793042E2032E8BD1254B1B6813F4003F03D07C
S315080079406368002B00F03382236813F0020F58D0C7
S31508007950042D45D00C2D41D0E368002B77D01B4A67
S31508007960136843F480731360FDF7B8FC0646174B9B
S315080079701B6813F4806F61D1FDF7B0FC801B0228E9
S31508007980F5D9032018E2114A136843F480331360CB
S315080079906FE703F18043A3F53C331A6842F480226B
S315080079A01A601A6842F480321A6062E7FDF796FC9C
S315080079B00746064B1B6813F4003FC5D0FDF78EFC3F
S315080079C0C01B6428F5D90320F6E100BF0010024069
S315080079D0CCD00008940000209C000020022EBBD1C9
S315080079E0A44B1B6813F4806F03D0E368002B00F0E8
S315080079F0E081A04A536823F0F853216943EA0163FA
S31508007A005360236813F0080F4CD063699BB3994AF7
S31508007A10D2F8943043F00103C2F89430FDF75EFCC7
S31508007A200646944BD3F8943013F0020F3AD1FDF77B
S31508007A3055FC801B0228F4D90320BDE18D4A536802
S31508007A4023F0F853216943EA01635360D9E7894A69
S31508007A50136823F480731360FDF740FC0646854BD4
S31508007A601B6813F4806FCCD0FDF738FC801B022806
S31508007A70F5D90320A0E17F4AD2F8943023F0010318
S31508007A80C2F89430FDF72AFC06467A4BD3F89430B0
S31508007A9013F0020F06D0FDF721FC801B0228F4D94B
S31508007AA0032089E1236813F0040F7AD0714B9B6D8C
S31508007AB013F0805F36D16F4B9A6D42F080529A650B
S31508007AC09B6D03F080530193019B01266A4B1B684B
S31508007AD013F4807F28D0A368012B39D0052B3FD01B
S31508007AE0644BD3F8902022F00102C3F89020D3F813
S31508007AF0902022F00402C3F89020A368002B3DD002
S31508007B00FDF7ECFB07465B4BD3F8903013F0020FFA
S31508007B1046D1FDF7E3FBC01B41F288339842F2D900
S31508007B20032049E10026D1E7534A136843F48073DA
S31508007B301360FDF7D3FB07464F4B1B6813F4807F92
S31508007B40C9D1FDF7CBFBC01B0228F5D9032033E1C9
S31508007B50484AD2F8903043F00103C2F89030CCE797
S31508007B60444BD3F8902042F00402C3F89020D3F88F
S31508007B70902042F00102C3F89020BEE7FDF7AEFB65
S31508007B8007463C4BD3F8903013F0020F08D0FDF7A8
S31508007B90A5FBC01B41F288339842F2D903200BE1BA
S31508007BA0E6B9236813F0200F35D0636AE3B1314A8A
S31508007BB0D2F8983043F00103C2F89830FDF78EFBEF
S31508007BC006462C4BD3F8983013F0020F23D1FDF755
S31508007BD085FB801B0228F4D90320EDE0254A936D26
S31508007BE023F080539365DCE7224AD2F8983023F0D5
S31508007BF00103C2F89830FDF771FB06461D4BD3F812
S31508007C00983013F0020F06D0FDF768FB801B022898
S31508007C10F4D90320D0E0A36A002B00F0CC80022B15
S31508007C2017D00C2D00F0CC80124A136823F080730D
S31508007C301360FDF753FB04460E4B1B6813F0007FD9
S31508007C4000F0A880FDF74AFB001B0228F4D90320A0
S31508007C50B2E0084BDB6803F00301E26A91420DD0FB
S31508007C600C2D00F0AB80034B1B6813F0806F2FD0F0
S31508007C700120A1E0001002400070004003F07002ED
S31508007C80216B0139B2EB011FEAD103F4FE42616BA5
S31508007C90B2EB012FE4D103F07842A16BB2EBC16FCE
S31508007CA0DED103F4C001E26B5208013AB1EB425F40
S31508007CB0D6D103F0C063226C5208013AB3EB426F87
S31508007CC0CED1404B1B6813F0007F49D0002073E0EB
S31508007CD03C4A136823F080731360FDF7FFFA0546E4
S31508007CE0384B1B6813F0007F06D0FDF7F7FA401BE8
S31508007CF00228F5D903205FE0324AD3683249194091
S31508007D00E36A206B013843EA0013606B43EA0023F9
S31508007D10E06B4008013843EA4053206C40080138BC
S31508007D2043EA4063A06B43EAC0631943D160136812
S31508007D3043F080731360D36843F08073D360FDF714
S31508007D40CDFA04461F4B1B6813F0007F06D1FDF7DA
S31508007D50C5FA001B0228F5D903202DE000202BE0E8
S31508007D60184B1A6842F080721A60DA6842F080721C
S31508007D70DA60FDF7B3FA0446124B1B6813F0007F6E
S31508007D8006D1FDF7ABFA031B022BF5D9032013E046
S31508007D90002011E00B4AD1680C4B0B40D360002041
S31508007DA00AE001207047012006E0012004E00120D6
S31508007DB002E0012000E0002003B0F0BD0120FBE74F
S31508007DC00120F9E7001002408C809D01FCFFEEFEC1
S31508007DD0002800F0AF8070B50D460446594B1B6865
S31508007DE003F007038B420BD2564A136823F00703A6
S31508007DF00B431360136803F007038B4240F09C8023
S31508007E00236813F0020F0CD0A2684F4B9B6803F04F
S31508007E10F0039A4205D94C498B6823F0F0031A43BC
S31508007E208A60236813F0010F39D06368032B09D0E1
S31508007E30022B26D063BB444A126812F0020F06D101
S31508007E40012076E0404A126812F0007F76D03E495B
S31508007E508A6822F0030213438B60FDF73FFA064651
S31508007E60394B9B6803F00C036268B3EB820F16D09C
S31508007E70FDF734FA801B41F288339842F0D9032083
S31508007E8057E0314A126812F4003FE0D1012050E071
S31508007E902D4A126812F4806FD9D1012049E023686F
S31508007EA013F0020F0CD0A268274B9B6803F0F0036F
S31508007EB09A4205D224498B6823F0F0031A438A6054
S31508007EC0204B1B6803F00703AB420AD91D4A136807
S31508007ED023F007032B431360136803F00703AB4231
S31508007EE02ED1236813F0040F06D0174A936823F49B
S31508007EF0E063E1680B439360236813F0080F07D02B
S31508007F00114A936823F46053216943EAC1039360D5
S31508007F10FFF7CEFB0C4B9B68C3F303130B4AD35CEA
S31508007F2003F01F03D8400A4B18600A4B1868FDF780
S31508007F3091F970BD012070470120FAE70120F8E7A2
S31508007F400120F6E70020024000100240CCD00008CD
S31508007F50940000209C000020F8B504460D46584BB6
S31508007F60DB6813F0030F17D0554BDB6803F00303E8
S31508007F700268934201D0012616E0002A00F09E808E
S31508007F804F4BDB68C3F3021301334268934201D0B7
S31508007F90012609E000261BE00368022B57D0032BB5
S31508007FA05CD0012B02D001263046F8BD444A12683F
S31508007FB012F0020F5ED04248C26822F0730261686E
S31508007FC0013943EA01131343C3600026002EEBD19F
S31508007FD03B4A136823F080631360FDF77FF9074671
S31508007FE0374B1B6813F0006F05D0FDF777F9C31BF5
S31508007FF0022BF5D90326002ED6D1002D3CD13049C7
S315080080000B6923F0784323F4FE43A068E268D2069E
S3150800801042EA002213430B61294A136843F080633E
S315080080201360FDF75BF90546254B1B6813F0006FD7
S3150800803005D1FDF753F9401B0228F5D90326002E72
S31508008040B2D11F4A1369A1690B431361ACE71C4AF5
S31508008050126812F4806FAED10126A5E7184A126895
S3150800806012F4003FA7D1164A126812F4802FA2D143
S31508008070012699E70126A9E7012D0FD010480269C4
S3150800808022F0C06222F4FE42A16863695B08013BE4
S315080080905B0643EA01231A430261BDE70848026901
S315080080A022F4C00222F4FE42A16823695B08013B60
S315080080B05B0543EA01231A430261ADE7012673E72C
S315080080C0001002402DE9F04182B00446036813F41B
S315080080D0006F25D0C36BB3F5000F06D0B3F5400F7C
S315080080E012D04BB1012637461CE0AE4AD36843F49A
S315080080F08033D360002708E000210430FFF72CFF07
S31508008100074610B106460DE00027A64AD2F8883081
S3150800811023F44003E16B0B43C2F88830002601E0E4
S3150800812000263746236813F4003F6BD09D4B9B6DA2
S3150800813013F0805F4CD19B4B9A6D42F080529A6542
S315080081409B6D03F080530193019B4FF00108964AFB
S31508008150136843F480731360FDF7C0F80546924B25
S315080081601B6813F4807F05D1FDF7B8F8401B022879
S31508008170F5D90327002F40D18A4BD3F8903013F452
S31508008180407315D0226D9A4212D0864AD2F89030A2
S3150800819023F44073D2F8901041F48031C2F890105D
S315080081A0D2F8901021F48031C2F89010C2F89030BD
S315080081B013F0010F0FD1002F40F0C980794AD2F889
S315080081C0903023F44073216D0B43C2F8903015E0CC
S315080081D04FF00008BBE7FDF781F80546714BD3F869
S315080081E0903013F0020FE6D1FDF778F8401B41F204
S315080081F088339842F2D90327DDE73E46B8F1000FE7
S3150800820040F0A780236813F0010F08D0654AD2F81A
S31508008210883023F00303216A0B43C2F888302368A9
S3150800822013F0020F08D05F4AD2F8883023F00C0307
S31508008230616A0B43C2F88830236813F0200F08D010
S31508008240584AD2F8883023F44063A16A0B43C2F82F
S315080082508830236813F4007F08D0524AD2F8883051
S3150800826023F44023616B0B43C2F88830236813F468
S31508008270806F08D04B4AD2F8883023F44013A16B9C
S315080082800B43C2F88830236813F0400F08D0454ADC
S31508008290D2F8883023F44053E16A0B43C2F8883099
S315080082A0236813F4807F08D03E4AD2F8883023F436
S315080082B04033216B0B43C2F88830236813F4005F00
S315080082C00FD0384AD2F8883023F04063216C0B432C
S315080082D0C2F88830236CB3F1006F40D0B3F1806FD9
S315080082E042D0236813F4802F0FD02E4AD2F8883054
S315080082F023F04063616C0B43C2F88830636CB3F1BA
S31508008300006F39D0B3F1806F3BD0236813F4804FE8
S315080083100CD0244AD2F8883023F04053A16C0B4382
S31508008320C2F88830A36CB3F1805F32D0236813F4A7
S31508008330004F08D01B4AD2F8883023F08043E16CFE
S315080083400B43C2F88830304602B0BDE8F0813E469D
S3150800835054E7144A936D23F08053936552E7D36824
S3150800836043F48013D360BCE70121201DFFF7F4FD19
S315080083700028B6D00646B4E7D36843F48013D36022
S31508008380C3E70121201DFFF7E7FD0028BDD00646FB
S31508008390BBE70221201DFFF7DFFD0028C6D00646F1
S315080083A0C4E700BF00100240007000402DE9F04706
S315080083B082B00546884617461E46FCF78FFF0A9B7D
S315080083C01B1A03EB0609FCF789FF8246284B1B6834
S315080083D0C3F3CB3309FB03F301932B689C6838EA94
S315080083E004040CBF01230023BB423DD0B6F1FF3F76
S315080083F0F3D0FCF773FFA0EB0A00484507D2019AB1
S3150800840002B14A46019B013B01939146E5E72A687A
S31508008410536823F0E00353606B68B3F5827F0BD093
S31508008420AB6AB3F5005F14D0012385F85D300023ED
S3150800843085F85C30032018E0AB68B3F5004F02D02E
S31508008440B3F5806FECD12A68136823F040031360F4
S31508008450E6E72A68136823F4005313602A6813684A
S3150800846043F400531360DFE7002002B0BDE8F0874D
S31508008470940000202DE9F04782B006460C461546C2
S315080084801F4600238DF80330FCF728FF0A9B1B1AAA
S3150800849003EB0708FCF722FF8146D6F800A0304B0D
S315080084A01B6803EB8303C3EBC3031B0D08FB03F332
S315080084B0019302E0B7F1FF3F12D133689B6803EAE4
S315080084C0040CAC4547D0B4F5C06FF3D1002DF1D1FB
S315080084D09AF80C30DBB28DF803309DF80330E9E7E3
S315080084E0FCF7FCFEA0EB0900404507D2019A02B151
S315080084F04246019B013B01939046DEE7326853688A
S3150800850023F0E00353607368B3F5827F0BD0B36A38
S31508008510B3F5005F14D0012386F85D30002386F892
S315080085205C30032018E0B368B3F5004F02D0B3F50A
S31508008530806FECD13268136823F040031360E6E7D6
S315080085403268136823F4005313603268136843F4DF
S3150800855000531360DFE7002002B0BDE8F08700BFD4
S315080085609400002070B582B004460D461646009267
S315080085700B4600224FF4C051FFF77CFFB0B90096B6
S315080085802B46002280212046FFF710FFA8B9009647
S315080085902B4600224FF4C0612046FFF76BFF50B10F
S315080085A0236E43F020032366032004E0236E43F082
S315080085B020032366032002B070BD236E43F0200318
S315080085C023660320F7E770B582B004460D461646C3
S315080085D04368B3F5827F0DD000962B460022802192
S315080085E02046FFF7E3FE90B96368B3F5827F14D09F
S315080085F002B070BD8368B3F5004F02D0B3F5806F43
S31508008600EAD12268136823F040031360E4E7236E77
S3150800861043F0200323660320EAE7A368B3F5004F77
S3150800862002D0B3F5806FE3D100962B4600224FF4B3
S31508008630C0612046FFF71EFF0028D9D0236E43F0FD
S31508008640200323660320D3E700286AD010B5044622
S31508008650436A33B94368B3F5827F05D00023C36103
S3150800866002E00023036143610023A36294F85D30AE
S31508008670002B4DD0022384F85D302268136823F05E
S3150800868040031360E368B3F5E06F47D90022B3F5FA
S31508008690706F04D0B3F5E06F01D00023A36263685E
S315080086A003F48273A16801F404410B43216901F0C4
S315080086B002010B43616901F001010B43A16901F451
S315080086C000710B43E16901F038010B43216A01F09F
S315080086D080010B43A16A01F4005120680B43036033
S315080086E0638B03F00403616A01F010010B43616BAD
S315080086F001F008010B43E16801F470610B4321683E
S315080087001A434A6000202066012384F85D3010BDB4
S3150800871084F85C302046FCF7A7FCABE74FF48052A0
S31508008720B5E701207047000038B5044690F85C00AC
S31508008730012800F0F780012084F85C0094F85D00B9
S31508008740C0B2656801280AD0B5F5827F40F0DB80A3
S31508008750A568002D40F0DC80042840F0DB80002965
S3150800876000F0DA80002A00F0D980002B00F0D880CB
S3150800877094F85D00C0B2042802D0052084F85D0094
S3150800878000202066A163A387E3872264A4F8443007
S31508008790A4F84630E06420652268536823F4C04391
S315080087A05360E368B3F5E06F28D92268536823F469
S315080087B08053536094F85D30DBB2042B69D0A36D07
S315080087C0594A1A63A36D594ADA62A36D584A5A631D
S315080087D0A36D00229A632168B4F846309BB2226CD6
S315080087E00C31A06DFEF784FA002859D0236E43F0A9
S315080087F010032366012084F85D0085E0226853682B
S3150800880043F480535360636D9B69B3F5806F1AD048
S31508008810A36D9B69B3F5806FCCD12268536823F4A6
S3150800882080535360B4F8463013F0010F24D1226800
S31508008830536823F400535360B4F84630C3F34E0329
S31508008840A4F84630B6E7A38F13F0010F09D12268C2
S31508008850536823F480435360E38FC3F34E03E387DF
S31508008860D6E72268536843F480435360E38FC3F323
S315080088704E030133E387CBE72268536843F400537A
S315080088805360B4F84630C3F34E030133A4F84630B8
S3150800889090E7A36D274A1A63A36D274ADA6294E71D
S315080088A02268536843F001035360626D0023136323
S315080088B0626DD362626D5363626D93632268E38F60
S315080088C09BB20C32A16B606DFEF712FA98B9236859
S315080088D01A6812F0400F03D11A6842F040021A6073
S315080088E02268536843F0200353602268536843F0B4
S315080088F00203536008E0236E43F010032366012049
S3150800890084F85D0000E00220002384F85C3038BD5E
S315080089100220F9E70220F7E70120F5E70120F3E74F
S315080089200120F1E70220F2E74B890008E7890008F1
S31508008930558900083F89000877890008704708B5F7
S31508008940806AFFF7FBFF08BD704708B5806AFFF726
S31508008950FBFF08BD08B5806A0268536823F0030365
S315080089605360036E43F010030366012380F85D30FD
S31508008970FBF73AFE08BD38B50546846AFCF7AEFC37
S315080089802B681B6813F0200F1FD1024621684B681D
S3150800899023F020034B60A3681BB96368B3F5827F95
S315080089A017D021684B6823F001034B6064212046E9
S315080089B0FFF709FE08B1202323660023A4F84630F2
S315080089C0012384F85D30236E4BB92046FBF7FAFD88
S315080089D038BD21684B6823F003034B60E6E7204661
S315080089E0FBF702FEF4E738B50546846AFCF776FC21
S315080089F02B681B6813F0200F1CD1024621684B68B0
S31508008A0023F020034B6064212046FFF7ABFD18B125
S31508008A10236E43F0200323662268536823F003037A
S31508008A2053600023E387A4F84630012384F85D30B9
S31508008A30236E1BB92046FBF7B3FD38BD2046FBF76E
S31508008A40D3FDFAE710B584B0044602685168936806
S31508008A5003F04100012867D013F0020F02D011F08D
S31508008A60800F68D113F4B07F68D011F0200F65D05D
S31508008A7013F0400F0FD094F85D00C0B203285FD002
S31508008A80206E40F00400206600200090D068009018
S31508008A9090680090009813F0200F0CD0206E40F0DC
S31508008AA0010020660020029090680290106820F06D
S31508008AB040001060029A13F4807F09D0236E43F0B9
S31508008AC0080323660023039323689B680393039B89
S31508008AD0236E002B32D02268536823F0E0035360DC
S31508008AE0012384F85D3011F0030F31D022685368F2
S31508008AF023F003035360A36D4BB1174A9A63A06D25
S31508008B00FEF731F918B1236E43F040032366636D0F
S31508008B10A3B1114A9A63606DFEF725F970B1236E09
S31508008B2043F04003236609E011F0400F94D0E36C4C
S31508008B302046984702E0236D2046984704B010BDAA
S31508008B4000230193D368019393680193019BF5E78A
S31508008B502046FBF749FDF1E75D8B000808B5806AFA
S31508008B600023A0F84630C387FBF73EFD08BD8446C0
S31508008B70002311208B4212D230B402E008338B4214
S31508008B800BD203EB0C02D2E90045B5F1FF3F08BF53
S31508008B90B4F1FF3FF2D01020F0E730BC70477047C1
S31508008BA02DE9F003D0E90089D0E90267D0E9044548
S31508008BB0D0E90623B3F1FF3F08BFB2F1FF3F13D157
S31508008BC0B5F1FF3F08BFB4F1FF3F11D1B7F1FF3F41
S31508008BD008BFB6F1FF3F0DD1B9F1FF3F08BFB8F1A5
S31508008BE0FF3F09D1002000E00420BDE8F0037047EC
S31508008BF00320FAE70220F8E70120F6E738B504462D
S31508008C0000F5803C4FEACC2C284BD3F8E02590B2EF
S31508008C104FF6FF73984215D0254B03EA82234FF48B
S31508008C20F032B2FBF3F203FB02CC0CF108050CF1AF
S31508008C3010000CF1180E0139032931D8DFE801F0CC
S31508008C4005101B254FF48023E9E74FF0AA324FF0B1
S31508008C50AA33604600F08AFF20BB164B1C7038BD4D
S31508008C604FF0AA324FF0AA33284600F07FFFD8B952
S31508008C70104B1C70F3E74FF0AA324FF0AA3300F0FE
S31508008C8075FF0028EBD00220E9E74FF0AA324FF033
S31508008C90AA33704600F06AFF0028E0D00220DEE71B
S31508008CA00020DCE70220DAE70220D8E70070FF1F81
S31508008CB000FCFF03E004002038B5054600F088FFF5
S31508008CC0002840F092804B4BD3F8E02591B24FF63E
S31508008CD0FF7399420CD0484B03EA82234FF4F034D1
S31508008CE0B4FBF3F403FB04F4C4F5F034E40A13E02C
S31508008CF04FF48023F2E704F580304FF4F033B3FBEA
S31508008D00F2F302FB03F34FF4006103EBC020FFF715
S31508008D102EFF102821D00134364BD3F8E03599B20E
S31508008D204FF6FF72914220D0334A02EA83224FF46B
S31508008D30F033B3FBF2F302FB03F3C3F5F033DB0ABC
S31508008D400433A34214D9002DD5D10121204600F0C1
S31508008D5019FF0028DFD0012040E00121204600F05D
S31508008D6011FF0028D7D0012038E04FF48022DEE733
S31508008D7000F01AFF1F4BD3F8E02591B24FF6FF73A8
S31508008D8099422CD01C4B03EA82234FF4F030B0FBF7
S31508008D90F3F003FB00F0C0F5F0300221C00AFFF73C
S31508008DA02DFF20BB154B00221A80124BD3F8E03555
S31508008DB099B24FF6FF72914214D00F4A02EA832203
S31508008DC04FF4F033B3FBF2F302FB03F3C3F5F033CE
S31508008DD0DB0A0B4A13700B4B20221A6038BD4FF47E
S31508008DE08023D2E74FF48022EAE70E20F6E7022036
S31508008DF0F4E700BF0070FF1F00FCFF03E204002039
S31508008E00E0040020C000002038B5394BD3F8E0252F
S31508008E1091B24FF6FF7399420CD0364B03EA822380
S31508008E204FF4F034B4FBF3F403FB04F4C4F5F03464
S31508008E30E40A4CE04FF48023F2E7651CA31CAB421E
S31508008E4007D80221204600F09DFE0446F0B1012411
S31508008E5049E005F58032D202254BD3F8E01588B2F1
S31508008E604FF6FF7398420ED0224B03EA81234FF444
S31508008E70F030B0FBF3F003FB0020FFF791FE042867
S31508008E8033D10135DAE74FF48023F0E700F08CFEA2
S31508008E9029E0184A02EA83224FF4F033B3FBF2F3CF
S31508008EA002FB03F3C3F5F033DB0A0433A34219D9F3
S31508008EB004F580304FF4F033B3FBF2F302FB03F30F
S31508008EC003EBC020FFF76CFE0428B6D00234084B2B
S31508008ED0D3F8E03599B24FF6FF729142D9D14FF4E3
S31508008EE08022D9E70524204638BD0524FBE700BFC4
S31508008EF00070FF1F00FCFF03F8B50646614B1D789E
S31508008F0005F58032D202604BD3F8E01588B24FF6E9
S31508008F10FF7398424FD05D4B03EA81234FF4F0303C
S31508008F20B0FBF3F003FB0020FFF73AFE0746564B6B
S31508008F30D3F8E03599B24FF6FF7291423ED0534AC4
S31508008F4002EA83224FF4F033B3FBF2F302FB03F396
S31508008F50C3F5F032A5EBD224013404F0030404EB84
S31508008F60D22404F5803003EBC020FFF719FE464BE8
S31508008F70D3F8E03599B24FF6FF72914221D0434AB1
S31508008F8002EA83224FF4F033B3FBF2F302FB03F356
S31508008F90C3F5F033A5EBD322033202F0030202EB4A
S31508008FA0D322012E10D0022E57D0002E4CD04FF0CF
S31508008FB0FF352846F8BD4FF48023AFE74FF48022EB
S31508008FC0C0E74FF48022DDE7022F19D0012F4DD1DB
S31508008FD02F4B1B68B3F5006FEBD304282DD0032164
S31508008FE02846FFF70BFE002843D101212046FFF74C
S31508008FF005FE002840D1264B20221A602546D8E7D0
S31508009000234B1B68B3F5006FD3D304280ED0032176
S315080090102846FFF7F3FD18BB02212046FFF7EEFDB1
S3150800902008BB1B4B20221A602546C2E7FFF7ECFE59
S315080090300028ECD04FF0FF35BBE7FFF7E5FE002828
S31508009040CDD04FF0FF35B4E7022FB2D0012F02D0B2
S315080090504FF0FF35ADE71546ABE780B92546A8E7DB
S315080090604FF0FF35A5E74FF0FF35A2E74FF0FF3584
S315080090709FE74FF0FF359CE74FF0FF3599E74FF034
S31508009080FF3596E7E00400200070FF1F00FCFF0391
S31508009090C000002082B00B4B9A6C42F480529A644E
S315080090A09B6C03F480530193019B074A48F205031E
S315080090B05361936823F0180343F00803936002B0E2
S315080090C0704700BF0010024000300240044B9A6807
S315080090D042F001029A6018601980186880B27047D9
S315080090E0003002402DE9F04780468A460020FFF707
S315080090F003FFB0F1FF3F63D0814600F58035ED02EE
S31508009100304BD3F8E02591B24FF6FF7399420CD055
S315080091102D4B03EA82234FF4F032B2FBF3F203FB42
S3150800912002552846FFF73CFD3EE04FF48023F2E760
S31508009130083C1F2C16D92B19D3E90067B7F1FF3F56
S3150800914008BFB6F1FF3FF3D0B1B24145F0D138467A
S31508009150FFF7BCFFB0EB164FEAD1CAF80070002043
S31508009160BDE8F087174BD3F8E02591B24FF6FF73A9
S31508009170994220D0144B03EA82234FF4F035B5FB0D
S31508009180F3F503FB05F5C5F5F033A9EBD32909F18A
S31508009190030909F0030909EBD32909F5803305EB1F
S315080091A0C3252846FFF7FCFC0238C0B2022805D8BA
S315080091B04FF4FF64BDE74FF48023DEE70720CFE7CF
S315080091C00320CDE70070FF1F00FCFF03431E9BB280
S315080091D04FF6FD72934201D90820704710B582B048
S315080091E00C460023019301A9FFF77CFF019B23602E
S315080091F002B010BD224B1B88B3F5FC7F39D270B57F
S3150800920006460D460120FFF777FEB0F1FF3F32D044
S3150800921000F58034E4021B4BD3F8E02591B24FF6F3
S31508009220FF73994220D0184B03EA82234FF4F03299
S31508009230B2FBF3F203FB024405B9C6B13146284630
S31508009240FFF744FF114B196846EA00422B4660189F
S3150800925000F08CFC88B90D4A136808331360084A75
S3150800926013880133138070BD4FF48023DEE7284648
S31508009270E8E7122070470320F5E70220F3E700BF6E
S31508009280E20400200070FF1F00FCFF03C00000205E
S31508009290F0B583B005460E46002301931746002A0B
S315080092A04CD10220FFF728FE0446B0F1FF3F00F03C
S315080092B031819E4B00221A809D4B18709D4B2022AF
S315080092C01A60002F3CD09C4BD3F8E03599B24FF684
S315080092D0FF7291423BD0994A02EA83224FF4F03357
S315080092E0B3FBF2F302FB03F3C3F5F032A4EBD2248B
S315080092F0033404F0030404EBD22404F5803003EBB2
S31508009300C020FFF74DFC022824D0042829D0012FBD
S3150800931040F00481032840F00381012F00F0A38068
S3150800932031462846FFF766FF002840F0FB807F4B52
S315080093301C88022C40F2E180023CCFE00120B1E714
S315080093400121FFF75BFC0028BDD00223DFE04FF4C4
S315080093508022C3E704212046FFF750FC002840F08E
S31508009360DB80754BD3F8E03599B24FF6FF72914220
S3150800937018D0724A02EA83224FF4F033B3FBF2F3B1
S3150800938002FB03F3C3F5F032A4EBD224033404F052
S31508009390030404EBD22404F5803003EBC020FFF766
S315080093A0FFFB20E04FF48022E6E704212046FFF782
S315080093B025FCF0B10223AAE04FF480224FF4F033E3
S315080093C0B3FBF2F302FB03F3C3F5F032A4EBD224AA
S315080093D0033404F0030404EBD22404F5803003EBD1
S315080093E0C020FFF7DDFBC31EDBB2012B95D803288F
S315080093F0DBD0514BD3F8E03599B24FF6FF72914264
S31508009400DAD04E4A02EA8322D8E74C4A02EA812297
S315080094104FF4F031B1FBF2F102FB01330344D3E917
S315080094200023B3F1FF3F08BFB2F1FF3F1DD03F4A0B
S315080094301388013313803F4A1368083313600830D2
S31508009440B0F5006F11D23A4B1B7803F58033DB0277
S31508009450394AD2F8E0158CB24FF6FF729442D4D14D
S315080094604FF48022D4E72020EAE7314B1C78002706
S315080094701EE04FF480224FF4F033B3FBF2F302FB05
S3150800948003F3C3F5F032A4EBD224033404F0030447
S3150800949004EBD22404F5803003EBC020FFF780FBF1
S315080094A003287FF43DAF214A1388FC331380013724
S315080094B0032F3FF635AF204BD3F8E03599B24FF678
S315080094C0FF729142D5D01D4A02EA8322D3E7019959
S315080094D03046FFF78FFE0346C8B90134062C0ED86E
S315080094E0A542FAD0A6B201A93046FFF7FBFD03460E
S315080094F00028ECD00728F0D009E00124EEE7022185
S315080095000B4B1878FFF77AFB70B94FF4807318463F
S3150800951003B0F0BD0423FAE70223F8E70A23F6E7C7
S315080095200A23F4E70223F2E70223F0E7E204002025
S31508009530E0040020C00000200070FF1F00FCFF03AD
S315080095402DE9F047054600F043FB002840F0DD8290
S315080095500446FFF79FFDBE4B01221A70BD4BD3F898
S31508009560E02591B24FF6FF7399420CD0BA4B03EA45
S3150800957082234FF4F037B7FBF3F703FB07F7C7F57A
S31508009580F037FF0A0CE04FF48023F2E71A18B349C4
S315080095900A6092ED007B0833B3F5006FF6D3013706
S315080095A0AC4BD3F8E02591B24FF6FF7399421AD027
S315080095B0A94B03EA82234FF4F036B6FBF3F603FB16
S315080095C006F6C6F5F036F60A321DBA420ED907F582
S315080095D080324FF4F030B0FBF3F003FB00F000EB01
S315080095E0C2200023D8E74FF48023E4E74FF00008B1
S315080095F0974B83F80080C2464746C14602E008F109
S3150800960001080136934BD3F8E03599B24FF6FF724D
S31508009610914228D0904A02EA83224FF4F033B3FBF2
S31508009620F2F302FB03F3C3F5F033DB0A191DB1426B
S315080096301CD906F580304FF4F033B3FBF2F302FB86
S3150800964003F303EBC020FFF7ABFA431EDBB2012B93
S31508009650D5D90328D5D1B9F1000F00D1B24609F101
S3150800966001093746CDE74FF48022D6E7B8F1000F57
S3150800967016D1B9F1000F4CD0AAEB0301033101F062
S3150800968003010B4403F580334FF4F030B0FBF2F0DE
S3150800969002FB00F000EBC320FFF782FA042814D07F
S315080096A06C4BD3F8E02591B24FF6FF73994235D04B
S315080096B0694B03EA82234FF4F036B6FBF3F603FB55
S315080096C006F6C6F5F036F60A42E0624BD3F8E03500
S315080096D099B24FF6FF72914218D05F4A02EA832286
S315080096E04FF4F033B3FBF2F302FB03F3C3F5F033A5
S315080096F0A7EBD320013000F00300012100EBD320B3
S31508009700FFF77CFA0028CBD00224FFE14FF4802231
S31508009710E6E70020FFF7D0FA0446F7E14FF4802386
S31508009720C9E74FF4802143E0B31A013303F003037A
S31508009730134403F580334FF4F030B0FBF1F001FB2E
S3150800974000F000EBC320FFF72BFA002852D00136B1
S31508009750404BD3F8E03599B24FF6FF72914257D095
S315080097603D4A02EA83224FF4F033B3FBF2F302FBDD
S3150800977003F3C3F5F033DB0A0433B3424BD906F5DA
S3150800978080304FF4F033B3FBF2F302FB03F303EB41
S31508009790C020FFF705FA0128D9D12E4BD3F8E035BA
S315080097A099B24FF6FF729142BBD02B4901EA832149
S315080097B04FF4F033B3FBF1F301FB03F3C3F5F033D6
S315080097C0DA0AB6EBD32FAFD0931CB342ACD0B31A98
S315080097D0033303F00303134403F580334FF4F030E7
S315080097E0B0FBF1F001FB00F000EBC320FFF7D8F95E
S315080097F00328ACD11A4B1E70012200210846FFF738
S3150800980047FDB0F5807F40F084814FF0010904E000
S315080098104FF48022A7E74FF000090E4BD3F8E02556
S3150800982091B24FF6FF7399420ED00B4B03EA82238F
S315080098304FF4F036B6FBF3F603FB06F6C6F5F0363C
S31508009840F60A4FF0000842E04FF48023F0E700BF25
S31508009850D80400200070FF1F00FCFF03DC04002072
S31508009860E0040020AF4BD3F8E03599B24FF6FF720B
S31508009870914255D0AC4A02EA83224FF4F033B3FB47
S31508009880F2F302FB03F3C3F5F033D90AB6EBD32F91
S3150800989002D08B1CB34246D1731A013303F003037B
S315080098A00B4403F580334FF4F030B0FBF2F002FBC3
S315080098B000F000EBC320FFF773F938B9B8F1000FD1
S315080098C040F02981994B1E7008F101080136954B25
S315080098D0D3F8E03599B24FF6FF72914237D0924AE3
S315080098E002EA83224FF4F033B3FBF2F302FB03F3ED
S315080098F0C3F5F033DB0A191DB1422BD906F58030C2
S315080099004FF4F033B3FBF2F302FB03F303EBC0208F
S31508009910FFF746F90228A5D00328D7D13746D5E759
S315080099204FF48022A9E7731A033303F003030B44A9
S3150800993003F580334FF4F030B0FBF2F002FB00F091
S3150800994000EBC320FFF72CF90328BFD1B6E74FF485
S315080099508022C7E7B8F1000F06D0754B00221A809F
S315080099602022744B1A602AE0DBB2FA1AD2B201320C
S3150800997002F003021344D8B26C4B18700221FFF7A9
S315080099803DF90028E9D00224C0E04FF480214FF4C5
S31508009990F030B0FBF1F001FB00331344D3E90001CA
S315080099A0B1F1FF3F08BFB0F1FF3F1CD060490B88FB
S315080099B001330B805F490B6808330B600832B2F538
S315080099C0006F10D2594B1B7803F58033DB025549DB
S315080099D0D1F8E00586B24FF6FF718E42D5D05249CE
S315080099E001EA8021D3E7514B1F7827E04FF4802204
S315080099F04FF4F033B3FBF2F302FB03F3C3F5F03392
S31508009A00DE0AB7EBD32F25D0B31CBB4222D0BF1B2F
S31508009A10033707F00307374407F580304FF4F03370
S31508009A20B3FBF2F302FB03F303EBC020FFF7B8F82E
S31508009A30032872D13E4A1388FC331380394BD3F876
S31508009A40E03599B24FF6FF729142CFD0364A02EA14
S31508009A508322CDE7354B1B789B1B013303F00303A9
S31508009A601E4406F580314FF4F033B3FBF2F302FBE4
S31508009A7003F303EBC12023E04FF40061FFF777F807
S31508009A80102829D0274BD3F8E03599B24FF6FF7244
S31508009A90914229D0244A02EA83224FF4F033B3FBD9
S31508009AA0F2F302FB03F3C3F5F032A6EBD226013636
S31508009AB006F0030606EBD22606F5803203EBC22033
S31508009AC0B74214D0002DD7D10121304600F05AF8FC
S31508009AD00028D7D0012419E00121304600F052F8B9
S31508009AE00028CFD0012411E04FF48022D5E700F0FA
S31508009AF05BF8B9F1000F09D100210846FFF77AFB98
S31508009B0068B1122802D0022400E00E242046BDE8DF
S31508009B10F0870C24FAE70A24F8E70A24F6E704464D
S31508009B20F4E700BF0070FF1F00FCFF03E0040020FD
S31508009B30E2040020C000002038B504460D46FFF7B1
S31508009B4059FB122800D038BD002229462046FFF7C7
S31508009B509FFBF8E708B5431E9BB24FF6FD7293428A
S31508009B6001D9082008BDFFF7E7FFFBE710B5014656
S31508009B7003484CF2FB3404610020FDF7FBF910BDE5
S31508009B800020024000B587B0002301930293059197
S31508009B9004900123039301A902A8FDF799FA00B1DD
S31508009BA0012007B05DF804FB084B1A6822F48062AE
S31508009BB01A601A6842F480521A601A6822F48052AF
S31508009BC01A601A6842F480621A60704700200240E0
S31508009BD00020704708B502F044FB10B102684068DF
S31508009BE0904708BDEFF305832BB9064B186828B9CB
S31508009BF001221A6070476FF0050070474FF0FF307A
S31508009C00704700BF340C0020EFF3058373B90A4B85
S31508009C101B68012B0DD110B50024084BDC77064BC9
S31508009C2002221A6001F0F0FB204610BD6FF0050015
S31508009C3070474FF0FF307047340C002000ED00E00D
S31508009C4008B5EFF3058343B901F068FF40B1022870
S31508009C5008D101F02FFC002006E06FF0050003E0B4
S31508009C60012001E04FF0FF3008BDF0B587B00024B1
S31508009C700594EFF3058474BB68B322B3156893693A
S31508009C8003B918235C1E372C49D8546814F0010F01
S31508009C9047D156696EB14FEA960C94682CB1D768CD
S31508009CA0A72F02D9176907B1C6B92CB14FF0FF34EF
S31508009CB00EE04FF0800CF0E7D4688CB9146994B1C3
S31508009CC04FF0FF3404E01546002418234FF0800CAB
S31508009CD0012C0AD0ACB1059807B0F0BD0124F7E70E
S31508009CE04FF0FF34F4E70024F2E714699268029211
S31508009CF0019400930B466246294601F017FB05902E
S31508009D00E9E705AA019200930B461FFA8CF2294649
S31508009D1001F047FB0128DED000230593DBE700208E
S31508009D20DAE70020D8E708B5EFF3058323B930B1A1
S31508009D3001F04EFD002008BD6FF00500FBE76FF04F
S31508009D400300F8E708B5EFF3058333B908B900202F
S31508009D5008BD01F0C5FC0020FAE76FF00500F7E73B
S31508009D602DE9F04383B0EFF30587002F43D106466C
S31508009D70894615461C4600283FD0082002F0BAFC42
S31508009D80804600283BD006604560B9F1000F00D038
S31508009D90012704B32068A36813B1E2682B2A10D8F8
S31508009DA053B14FF0FF33DBB10024404602F024FDE7
S31508009DB0204603B0BDE8F083E3687BB14FF0FF337C
S31508009DC0F1E701930F4B009343463A46012102F00F
S31508009DD093F804460CE020460023E4E70023E2E774
S31508009DE0084B009343463A46012102F069F80446B7
S31508009DF0002CDDD1D9E70024DAE70024D8E70446A9
S31508009E00D6E700BFD59B0008EFF305836BB90A4672
S31508009E1070B100B583B00093042102F097F80128C9
S31508009E2009D1002003B05DF804FB6FF00500704708
S31508009E306FF0030070476FF00200F3E708B5EFF321
S31508009E400583CBB9A0B1836813B1C2681F2A0BD8A2
S31508009E502BB14FF0FF338BB900F050FA08BDC36839
S31508009E6043B14FF0FF33F6E7184600F022FAF5E75C
S31508009E700023F0E70023EEE70020EFE70020EDE7F8
S31508009E80F8B110B582B00C46B1F1807F1CD2EFF361
S31508009E9005829AB10022019201AA00F04DFBB8B1E1
S31508009EA0019BC3B14FF0E0234FF08052C3F8042D55
S31508009EB0BFF34F8FBFF36F8F204607E000F0F0FA2D
S31508009EC004E06FF0030070476FF0030002B010BDA6
S31508009ED06FF00200FAE72046F8E770B5B0B10C4615
S31508009EE00646B1F1807F14D2EFF3058353B100F033
S31508009EF0C9FA05462146304600F0BAFA58B96FF055
S31508009F00020508E000F08DFA054604E06FF0030547
S31508009F1001E06FF00305284670BD40B370B582B006
S31508009F200C461D468446B1F1807F23D2EFF30583A4
S31508009F3023BB12F0010610D0012312F0020F0ED037
S31508009F40002200952146604600F0E6F94EB18443AA
S31508009F5012D0B5B16FF001000EE00023EDE7012243
S31508009F60EFE7044208D17DB16FF0010004E06FF01D
S31508009F70030070476FF0030002B070BD6FF0050074
S31508009F80FAE76FF00200F7E76FF00200F4E770B542
S31508009F90EFF30583002B3CD1044600B1436813F068
S31508009FA0010600D0012613F0080F35D144B3A16885
S31508009FB011B1E3684F2B18D891B14FF0FF336BBB43
S31508009FC016B3042000F040FD05461DB304B124680D
S31508009FD02146284600F0D2FFE6B145F0010519E012
S31508009FE0E3687BB14FF0FF33E9E726B1042000F0C0
S31508009FF036FD0546E9E7012000F031FD0546E4E7B0
S3150800A0000023DCE70023DAE7012000F01DFD054602
S3150800A010DBE70025284670BD0025FBE70025F9E7A4
S3150800A020EFF30582DAB910B503460C4620F00100B5
S3150800A03003F00101012B15D941B1214600F027FF94
S3150800A040012812D09CB16FF001000FE0214600F004
S3150800A0504BFE01280ED07CB16FF0010006E06FF0D0
S3150800A060050070476FF0030000E0002010BD6FF098
S3150800A0700200FBE70020F9E76FF00200F6E7EFF3CE
S3150800A0800582BAB908B5034620F0010003F00101BC
S3150800A090012B12D929B100F0F1FC012810D10020BA
S3150800A0A008BD00231A46194600F0FEFB01280AD10E
S3150800A0B00020F5E76FF0050070476FF00300EFE743
S3150800A0C06FF00200ECE76FF00200E9E770B582B0C6
S3150800A0D0EFF30583002B3AD1144600283BD000291C
S3150800A0E03BD06AB393684BB1D2684F2A06D9226926
S3150800A0F022B101FB00F56669AE421BD273B14FF07F
S3150800A100FF3363BB002200F0ABFB054605B304B181
S3150800A11024682146284600F031FF19E0E3688BB928
S3150800A120236913B14FF0FF33EBE763696BB14FF067
S3150800A130FF33E6E70025009500F048FB0546E5E70E
S3150800A1400023DEE74FF0FF33DBE70023D9E70025DE
S3150800A150284602B070BD0025FAE70025F8E7002575
S3150800A160F6E710B582B01C46EFF30583C3B118B302
S3150800A17029B33CBB0023019301AA00F09FFC0128E8
S3150800A18023D1019850B14FF0E0234FF08052C3F825
S3150800A190042DBFF34F8FBFF36F8F002002B010BDA1
S3150800A1A0B0B1C1B10023224600F07EFB012815D0CC
S3150800A1B0B4B16FF00100F1E76FF00300EEE76FF05E
S3150800A1C00300EBE76FF00300E8E76FF00200E5E74E
S3150800A1D06FF00300E2E76FF00300DFE70020DDE73A
S3150800A1E06FF00200DAE710B582B01C46EFF305837C
S3150800A1F0C3B110B321B334BB0023019301AA00F005
S3150800A20066FE012822D1019850B14FF0E0234FF0A5
S3150800A2108052C3F8042DBFF34F8FBFF36F8F002012
S3150800A22002B010BDA8B1B9B1224600F0AEFC0128B3
S3150800A23015D0B4B16FF00100F2E76FF00300EFE755
S3150800A2406FF00300ECE76FF00300E9E76FF0020038
S3150800A250E6E76FF00300E3E76FF00300E0E70020AE
S3150800A260DEE76FF00200DBE7034B0360034B0B608E
S3150800A27080231360704700BF8C0B00208C090020D8
S3150800A280034B0360034B0B604FF4807313607047F6
S3150800A290E4080020E40400201AB9084205D1104653
S3150800A2A07047814303D00020704701207047012082
S3150800A2B0704780B110B582B0044620230193019BF4
S3150800A2C0202B11D04FF0500383F31188BFF36F8F03
S3150800A2D0BFF34F8FFEE74FF0500383F31188BFF3A8
S3150800A2E06F8FBFF34F8FFEE7002340F8043B00F063
S3150800A2F02DF901232377204602B010BD38B520205A
S3150800A30002F0F8F9044628B1002540F8045B00F08D
S3150800A3101DF92577204638BD88B12DE9F0410C4650
S3150800A32016461D460746B1F1807F11D34FF05003FC
S3150800A33083F31188BFF36F8FBFF34F8FFEE74FF09C
S3150800A340500383F31188BFF36F8FBFF34F8FFEE778
S3150800A35041B94FF0500383F31188BFF36F8FBFF3F2
S3150800A3604F8FFEE701F0DAFB50B9069B43B14FF079
S3150800A370500383F31188BFF36F8FBFF34F8FFEE748
S3150800A38001F098F8D7F800802A4621464046FFF79C
S3150800A39083FFF8B18EB328EA04033B6000230693D3
S3150800A3A001F022F9069B93B148B94FF0E0234FF02C
S3150800A3B08052C3F8042DBFF34F8FBFF36F8F01F0A0
S3150800A3C0A1FC804610F0007F1AD028F07F4840464E
S3150800A3D0BDE8F081069B002BE2D05EB900210DB1E5
S3150800A3E041F08061069A2143381D01F06BFA4FF05F
S3150800A3F00008D5E74FF08071F1E700230693CFE711
S3150800A40001F0C0FFD7F800802A4621464046FFF7EC
S3150800A41043FF18B116B128EA04043C6001F0D4FFE2
S3150800A420D3E770B170B50C460546B1F1807F11D3FC
S3150800A4304FF0500383F31188BFF36F8FBFF34F8F2D
S3150800A440FEE74FF0500383F31188BFF36F8FBFF316
S3150800A4504F8FFEE701F096FF2E6826EA04042C606B
S3150800A46001F0B2FF304670BD08B5FFF7DAFF08BD48
S3150800A47008B50A4600230146014801F005FF08BD54
S3150800A48069A40008EFF311834FF0500282F3118894
S3150800A490BFF36F8FBFF34F8F006883F31188704740
S3150800A4A0F8B568B10D460446B1F1807F11D34FF077
S3150800A4B0500383F31188BFF36F8FBFF34F8FFEE707
S3150800A4C04FF0500383F31188BFF36F8FBFF34F8F9D
S3150800A4D0FEE700F10C0600F0EDFF206923682B4328
S3150800A4E0236000270AE0216832EA010105D111E05C
S3150800A4F0216841F0007101F073FA2846B0420ED087
S3150800A5004568036823F07F4213F0806FEBD121681A
S3150800A5101142F2D013F0807FEAD01743E8E72368A8
S3150800A52023EA0703236001F05FF82068F8BD08B541
S3150800A530FFF7B6FF08BD000008B513460A460146F0
S3150800A540014801F0A1FE08BD2FA5000800F1080387
S3150800A55043604FF0FF328260C360036100230360EB
S3150800A560704700230361704743684B609A688A60A6
S3150800A570516099600861036801330360704730B41D
S3150800A5800D68B5F1FF3F11D000F108031C465B6862
S3150800A5901A68AA42FAD963684B6099608C60616050
S3150800A5A0086103680133036030BC70470469F2E749
S3150800A5B00369416882688A60416851605A688242C4
S3150800A5C006D0002202611A68013A1A6018687047B4
S3150800A5D082685A60F5E70346406A18B11B6B18682B
S3150800A5E0C0F13800704710B5044601F0CBFEA26BE7
S3150800A5F0E36B9A4204D0002401F0E6FE204610BD23
S3150800A6000124F9E710B5044601F0BCFEA36B23B993
S3150800A610012401F0D9FE204610BD0024F9E770B5E3
S3150800A62004461546866B026C5AB903681BB10020AE
S3150800A6300136A66370BD806801F0CCFA0023A360DA
S3150800A640F6E76DB9406802F0C3F96368226C1344F3
S3150800A6506360A268934219D3236863602846E7E7D4
S3150800A660C06802F0B5F9E368226C51429B1AE360B0
S3150800A6702268934202D2A3680B44E360022D01D0FC
S3150800A6800020D5E726B1013E0020D1E72846CFE7CE
S3150800A6900020CDE70346026C6AB110B50846D968B2
S3150800A6A01144D9609C68A14201D31968D960D96858
S3150800A6B002F08EF910BD704738B5054601F062FE06
S3150800A6C095F8454064B201E0013C64B2002C0ADD0D
S3150800A6D06B6A43B105F1240001F03CF90028F3D078
S3150800A6E001F010FAF0E7FF2385F8453001F06CFE1B
S3150800A6F001F048FE95F8444064B201E0013C64B2BA
S3150800A700002C0ADD2B6943B105F1100001F022F98E
S3150800A7100028F3D001F0F6F9F0E7FF2385F8443076
S3150800A72001F052FE38BD38B5E0B10D46044601F0D9
S3150800A73029FE2368E26B216C01FB0230A060002031
S3150800A740A0636360013A02FB0133E360FF2384F8E8
S3150800A750443084F84530FDB9236963B901F034FE05
S3150800A760012038BD4FF0500383F31188BFF36F8F74
S3150800A770BFF34F8FFEE704F1100001F0EBF8002855
S3150800A780ECD04FF0E0234FF08052C3F8042DBFF30E
S3150800A7904F8FBFF36F8FE1E704F11000FFF7D6FE86
S3150800A7A004F12400FFF7D2FED8E738B51D46049C0D
S3150800A7B00B4649B92460E063236401212046FFF76C
S3150800A7C0B2FF84F84C5038BD2260F4E740B94FF028
S3150800A7D0500383F31188BFF36F8FBFF34F8FFEE7E4
S3150800A7E010B584B01C46844653B192B189B94FF06E
S3150800A7F0500383F31188BFF36F8FBFF34F8FFEE7C4
S3150800A8004FF0500383F31188BFF36F8FBFF34F8F59
S3150800A810FEE76AB150230393039B502B13D04FF0E6
S3150800A820500383F31188BFF36F8FBFF34F8FFEE793
S3150800A8300029EFD04FF0500383F31188BFF36F8FD1
S3150800A840BFF34F8FFEE7039B012384F8463000943D
S3150800A8509DF818306046FFF7A8FF204604B010BDE3
S3150800A86040B94FF0500383F31188BFF36F8FBFF3DE
S3150800A8704F8FFEE7F0B583B00D461446064601FB3A
S3150800A88000F0503001F036FF074650B1002380F83B
S3150800A89046300090234600F1500229463046FFF71D
S3150800A8A084FF384603B0F0BDF0B585B0019288B193
S3150800A8B00F461D460446B1B1022D20D1E36B012B8C
S3150800A8C01DD04FF0500383F31188BFF36F8FBFF38A
S3150800A8D04F8FFEE74FF0500383F31188BFF36F8F56
S3150800A8E0BFF34F8FFEE7036C002BE5D04FF0500304
S3150800A8F083F31188BFF36F8FBFF34F8FFEE701F025
S3150800A9000DF9064658B9019B002B48D04FF0500365
S3150800A91083F31188BFF36F8FBFF34F8FFEE70026CF
S3150800A9203DE02A4639462046FFF779FE636A7BB939
S3150800A93048B14FF0E0234FF08052C3F8042DBFF31F
S3150800A9404F8FBFF36F8F01F03FFD012005B0F0BDBB
S3150800A95004F1240000F0FEFF0028F4D04FF0E023B5
S3150800A9604FF08052C3F8042DBFF34F8FBFF36F8F9C
S3150800A970E9E701F029FD0020E8E702A801F074F8EC
S3150800A980012619E0002384F8443021E0002384F8E6
S3150800A990453023E02046FFF78FFE00F025FE01F044
S3150800A9A0F1FCA26BE36B9A42BBD3022DB9D0019B93
S3150800A9B0002BDED0002EE0D001F006FD00F07AFD77
S3150800A9C001F0E0FC94F8442052B2B2F1FF3FD9D02E
S3150800A9D094F8452052B2B2F1FF3FD7D001F0F4FC0B
S3150800A9E001A902A801F04CF8D8B92046FFF7FBFDEB
S3150800A9F00028CFD0019904F1100000F04BFF204643
S3150800AA00FFF75AFE00F0F0FD0028C8D14FF0E0230A
S3150800AA104FF08052C3F8042DBFF34F8FBFF36F8FEB
S3150800AA20BDE72046FFF748FE00F0DEFD00208DE773
S3150800AA3048B108B5002181600160C1600B460A462D
S3150800AA40FFF732FF08BD704710B502460021012006
S3150800AA50FFF706FF0446FFF7EBFF204610BD10B5CB
S3150800AA6082B00B460090002211460120FFF7AEFE89
S3150800AA700446FFF7DDFF204602B010BD38B538B1F1
S3150800AA800446856801F044F885420AD0002038BD9E
S3150800AA904FF0500383F31188BFF36F8FBFF34F8FC7
S3150800AAA0FEE7E368013BE3600BB10120EFE71A46D6
S3150800AAB019462046FFF7F8FE0120E8E72DE9F84396
S3150800AAC090B10F4616461C460546B1B1022C20D158
S3150800AAD0EB6B012B1DD04FF0500383F31188BFF3A6
S3150800AAE06F8FBFF34F8FFEE74FF0500383F3118844
S3150800AAF0BFF36F8FBFF34F8FFEE7036C002BE5D0D4
S3150800AB004FF0500383F31188BFF36F8FBFF34F8F56
S3150800AB10FEE701F05DFDEFF311884FF0500383F374
S3150800AB201188BFF36F8FBFF34F8FAA6BEB6B9A42F7
S3150800AB3006D3022C04D0002088F31188BDE8F883D8
S3150800AB4095F845904FFA89F9AB6B2246394628465F
S3150800AB50FFF765FDB9F1FF3F06D009F101035BB2C6
S3150800AB6085F845300120E7E76B6A0BB90120E3E772
S3150800AB7005F1240000F0EEFE18B126B10120306080
S3150800AB80DAE70120D8E70120D6E7F0B585B00192CB
S3150800AB9090B10F460446C1B100F0C0FF064600BB9F
S3150800ABA0019B002B5ED04FF0500383F31188BFF34F
S3150800ABB06F8FBFF34F8FFEE74FF0500383F3118873
S3150800ABC0BFF36F8FBFF34F8FFEE7036C002BE3D005
S3150800ABD04FF0500383F31188BFF36F8FBFF34F8F86
S3150800ABE0FEE700263EE039462046FFF753FD013DC5
S3150800ABF0A563236923B901F0E7FB012005B0F0BD81
S3150800AC0004F1100000F0A6FE0028F4D04FF0E0236F
S3150800AC104FF08052C3F8042DBFF34F8FBFF36F8FE9
S3150800AC20E9E701F0D1FB0020E8E702A800F01CFFE5
S3150800AC30012621E0002384F8443029E0002384F823
S3150800AC4045302BE02046FFF737FD00F0CDFC09E044
S3150800AC502046FFF731FD00F0C7FC2046FFF7D2FC7F
S3150800AC6000283FD101F08EFBA56B002DBBD1019BBF
S3150800AC70002BD6D0002ED8D001F0A6FB00F01AFC87
S3150800AC8001F080FB94F844305BB2B3F1FF3FD1D0BA
S3150800AC9094F845305BB2B3F1FF3FCFD001F094FB97
S3150800ACA001A902A800F0ECFE0028D1D12046FFF742
S3150800ACB0A9FC0028C6D0019904F1240000F0EAFD99
S3150800ACC02046FFF7F9FC00F08FFC0028CAD14FF0A8
S3150800ACD0E0234FF08052C3F8042DBFF34F8FBFF324
S3150800ACE06F8FBFE7002089E770B584B0019158B12E
S3150800ACF00446036C8BB14FF0500383F31188BFF3FE
S3150800AD006F8FBFF34F8FFEE74FF0500383F3118821
S3150800AD10BFF36F8FBFF34F8FFEE700F0FFFE0546C8
S3150800AD2050B9019B5BB14FF0500383F31188BFF311
S3150800AD306F8FBFF34F8FFEE70026354655E0064670
S3150800AD4053E0013BA36323683BB123694BB901F088
S3150800AD503BFB0126304604B070BD00F0DFFFA06063
S3150800AD60F3E704F1100000F0F5FD0028EFD04FF0EE
S3150800AD70E0234FF08052C3F8042DBFF34F8FBFF383
S3150800AD806F8FE4E746B14FF0500383F31188BFF3A2
S3150800AD906F8FBFF34F8FFEE701F016FBDAE702A8C5
S3150800ADA000F062FE01252AE0002384F8443032E0F0
S3150800ADB0002384F8453034E001F0E4FAA06800F096
S3150800ADC0BDFE064601F000FB3BE02046FFF774FC9B
S3150800ADD000F00AFC09E02046FFF76EFC00F004FCD0
S3150800ADE02046FFF70FFC002842D101F0CBFAA36BEF
S3150800ADF0002BA6D1019B002BC4D0002DCFD001F08B
S3150800AE00E3FA00F057FB01F0BDFA94F844305BB260
S3150800AE10B3F1FF3FC8D094F845305BB2B3F1FF3FBA
S3150800AE20C6D001F0D1FA01A902A800F029FE00282F
S3150800AE30D1D12046FFF7E6FB0028C6D02368002BB1
S3150800AE40BAD0019904F1240000F024FD2046FFF74A
S3150800AE5033FC00F0C9FB0028C7D14FF0E0234FF0C0
S3150800AE608052C3F8042DBFF34F8FBFF36F8FBCE733
S3150800AE700EB900266EE701F085FA2046FFF7ABFB10
S3150800AE800146A06800F0EEFE01F09EFAF1E780B1F7
S3150800AE9070B50C460546866800F03AFE864211D023
S3150800AEA021462846FFF720FF80B1EB680133EB60A7
S3150800AEB00CE04FF0500383F31188BFF36F8FBFF395
S3150800AEC04F8FFEE7EB680133EB60012070BD2DE97B
S3150800AED0F843B0B10D4690460446D9B101F078FB67
S3150800AEE0EFF311874FF0500383F31188BFF36F8F89
S3150800AEF0BFF34F8FA66BCEB9002087F31188BDE844
S3150800AF00F8834FF0500383F31188BFF36F8FBFF3B5
S3150800AF104F8FFEE7036C002BE0D04FF0500383F30E
S3150800AF201188BFF36F8FBFF34F8FFEE794F84490F5
S3150800AF304FFA89F929462046FFF7ACFB731EA3632F
S3150800AF40B9F1FF3F06D009F101035BB284F844303A
S3150800AF500120D2E723690BB90120CEE704F11000DE
S3150800AF6000F0F8FC30B1B8F1000F05D00120C8F8A0
S3150800AF700000C2E70120C0E70120BEE70023072B37
S3150800AF800CD8074A52F833200AB10133F7E7044AC6
S3150800AF9042F8331002EBC30250607047704700BF97
S3150800AFA0380C002070B504460D46164601F0EAF93D
S3150800AFB094F844305BB2B3F1FF3F0DD094F84530B6
S3150800AFC05BB2B3F1FF3F0BD001F0FEF9A36B5BB1A7
S3150800AFD02046FFF771FB70BD002384F84430EDE787
S3150800AFE0002384F84530EFE73246294604F1240069
S3150800AFF000F094FCECE70000084B1B681B6823B9BB
S3150800B000074B4FF0FF321A607047044B1B68DB682A
S3150800B010DB685A68024B1A60704700BFE80C0020CC
S3150800B020800C00202DE9F04780460D4617469946C4
S3150800B030089EDDF824A00A9C9200A521206B01F049
S3150800B04042FC236B07F18042013A03EB820727F0A3
S3150800B0500707002D42D04FF0000CBCF10F0F09D89E
S3150800B06015F80C3004EB0C0282F8343013B10CF1ED
S3150800B070010CF2E7002384F84330372E00D937262F
S3150800B080E662E66400252565201DFFF76AFA04F1E5
S3150800B0901800FFF766FA2461C6F13806A6616462ED
S3150800B0A0C4F8A05084F8A4504C22294604F1540050
S3150800B0B001F009FC0B4BA36503F16802E265D03386
S3150800B0C023664A464146384601F030F92060BAF10F
S3150800B0D0000F01D0CAF80040BDE8F087002384F8C5
S3150800B0E03430CAE7CC92002038B5002407E004EBD8
S3150800B0F0840293000E481844FFF728FA0134372CC7
S3150800B100F5D90C4D2846FFF721FA0B4C2046FFF7D8
S3150800B1101DFA0A48FFF71AFA0948FFF717FA094805
S3150800B120FFF714FA084B1D60084B1C6038BD00BFBA
S3150800B130140D0020000D0020EC0C0020D00C00207F
S3150800B140BC0C0020A40C0020E80C0020E40C002015
S3150800B15010B5044601F016F9224A13680133136044
S3150800B160214B1B685BB1214B1B686BB91E4B1B68D7
S3150800B170DA6AE36A9A4207D81B4B1C6004E01A4B4A
S3150800B1801C601368012B29D0194A13680133136010
S3150800B1906364E06A174B1B68984201D9154B18601F
S3150800B1A000EB8000211D144B03EB8000FFF7DCF950
S3150800B1B001F00AF90D4B1B687BB10B4B1B68DA6A69
S3150800B1C0E36A9A4209D24FF0E0234FF08052C3F85F
S3150800B1D0042DBFF34F8FBFF36F8F10BDFFF784FFAA
S3150800B1E0D2E700BFA00C002074110020940C0020A8
S3150800B1F0840C0020980C0020140D002010B504467D
S3150800B200543001F069FB94F8A53063B1012B11D0D5
S3150800B210022B0ED04FF0500383F31188BFF36F8FC4
S3150800B220BFF34F8FFEE7206B01F0E6FA204601F0E8
S3150800B230E3FA10BD204601F0DFFAFAE70F4B1B6868
S3150800B240D3B110B501F09EF80D4BDB68DC68201D04
S3150800B250FFF7AEF90B4A1368013B1360074A1368F8
S3150800B260013B136001F0B0F82046FFF7C7FF034B18
S3150800B2701B68002BE6D110BD704700BFB80C002034
S3150800B280BC0C0020A00C002008B5FFF7D7FF074B21
S3150800B2901B68012BF9D94FF0E0234FF08052C3F811
S3150800B2A0042DBFF34F8FBFF36F8FEEE7140D002009
S3150800B2B070B504460D46174B1E68174B18680430C0
S3150800B2C0FFF776F9B4F1FF3F0DD03444124B1B68F3
S3150800B2D05C60A64210D9114B18680F4B19680431E7
S3150800B2E0FFF74DF970BD002DEFD00B4B19680431EF
S3150800B2F00B48FFF739F9F5E70A4B1868064B196842
S3150800B3000431FFF73CF9084B1B68A342EAD9064B00
S3150800B3101C60E7E79C0C002074110020E40C002058
S3150800B320A40C0020E80C0020800C002030B587B063
S3150800B3300B9C7CB10C9DB5B1A8250495049DA82D40
S3150800B3401AD04FF0500383F31188BFF36F8FBFF302
S3150800B3504F8FFEE74FF0500383F31188BFF36F8FCB
S3150800B360BFF34F8FFEE74FF0500383F31188BFF307
S3150800B3706F8FBFF34F8FFEE7049D0C9D2C6302244D
S3150800B38085F8A54000240394029505AC01940A9C0F
S3150800B3900094FFF747FE0C98FFF7DAFE059807B00A
S3150800B3A030BD2DE9F04385B00746884614461E464B
S3150800B3B0900001F09FF908B38146A82001F09AF998
S3150800B3C00546A8B1C0F83090002380F8A53003934D
S3150800B3D002900D9B01930C9B0093334622464146EF
S3150800B3E03846FFF71FFE2846FFF7B2FE012007E0A2
S3150800B3F0484601F001FA4FF0FF3001E04FF0FF3008
S3150800B40005B0BDE8F083000010B588B000240594A7
S3150800B410069407AA06A905A8FEF726FF059B029328
S3150800B420069B019300942346079A1A491A48FFF780
S3150800B4307DFF1A4B1860E8B100F010FD01281AD1FB
S3150800B4404FF0500383F31188BFF36F8FBFF34F8F0D
S3150800B450134B1B685433134A1360134B4FF0FF32D8
S3150800B4601A60124B01221A60114B00221A6001F071
S3150800B47023F803E00020B0F1FF3F01D008B010BD6B
S3150800B4804FF0500383F31188BFF36F8FBFF34F8FCD
S3150800B490FEE700BFDCD0000889B200087C0C00205B
S3150800B4A074110020C8000020800C0020940C002095
S3150800B4B09C0C0020024A136801331360704700BFD2
S3150800B4C0780C0020014B1868704700BF9C0C0020C0
S3150800B4D0F8B53A4B1B68002B69D1394B1D68013505
S3150800B4E01D60C5B9374B1B681B6843B14FF0500345
S3150800B4F083F31188BFF36F8FBFF34F8FFEE7314A8F
S3150800B5001168314B186810601960304A13680133A6
S3150800B5101360FFF771FD2E4B1B68AB423DD9002720
S3150800B5202C4B1B68DB6A03EB83039A002A4B9B5858
S3150800B530012B00D90127294B1B68002B3CD001277A
S3150800B5403AE001271F4B1B681B6843B31D4B1B685A
S3150800B550DB68DC6863689D4226D3261D3046FFF704
S3150800B56027F8A36A1BB104F11800FFF721F8E36A6C
S3150800B5701B4A1268934201D9194A136003EB8303E5
S3150800B5809A00314614481044FEF7EEFFE26A114B62
S3150800B5901B68DB6A9A42D4D2D4E70027D2E70C4B61
S3150800B5A04FF0FF321A60BBE7094A1360B8E70D4A45
S3150800B5B013680133136000273846F8BD780C00205D
S3150800B5C09C0C0020E80C0020E40C0020880C0020CD
S3150800B5D0800C002074110020140D00208C0C002013
S3150800B5E0980C0020900C002038B5354B1B6843B9E1
S3150800B5F04FF0500383F31188BFF36F8FBFF34F8F5C
S3150800B600FEE700F0BFFE2E4B1A68013A1A601B6867
S3150800B610002B4FD12B4B1B680BB900244BE00024A1
S3150800B620294B1B681BB3284BDB68DC6804F1180040
S3150800B630FEF7BEFF251D2846FEF7BAFFE06A234B34
S3150800B6401B68984201D9214B186000EB80002946F7
S3150800B6501F4B03EB8000FEF787FFE26A1D4B1B6852
S3150800B660DB6A9A42DCD31C4B01221A60D8E70CB17C
S3150800B670FFF7C2FC194B1C6884B9174B1C68D4B178
S3150800B6804FF0E0234FF08052C3F8042DBFF34F8FDD
S3150800B690BFF36F8F01240EE0013C07D0FFF718FFB8
S3150800B6A00028F9D00C4B01221A60F5E70B4B002253
S3150800B6B01A60E2E7002400F087FE204638BD00BF86
S3150800B6C0780C0020A00C0020D00C0020980C00203C
S3150800B6D0140D0020741100208C0C0020900C002002
S3150800B6E010B5A8B10446104B1B6843B14FF0500380
S3150800B6F083F31188BFF36F8FBFF34F8FFEE7FFF712
S3150800B700D9FE00212046FFF7D3FDFFF76DFF48B9A4
S3150800B7104FF0E0234FF08052C3F8042DBFF34F8F4C
S3150800B720BFF36F8F10BD00BF780C0020224B1B683B
S3150800B7301BB1224B01221A607047204B00221A6067
S3150800B7401F4B1B6803EB83018A001E498A585AB9A6
S3150800B7500BB1013BF6E74FF0500383F31188BFF3B3
S3150800B7606F8FBFF34F8FFEE7084603EB83018A000E
S3150800B770024451684968516003EB830C4FEA8C0216
S3150800B7800832024491420FD003EB830291000D4A1E
S3150800B7900A445268D1680C4A116009490B6013685B
S3150800B7A054330A4A13607047486862469100054A4E
S3150800B7B00A445060E8E700BF780C00208C0C002093
S3150800B7C0980C0020140D002074110020C8000020D9
S3150800B7D038B5044600F0D6FDE4B1251D2846FEF727
S3150800B7E0E7FEA36A1BB104F11800FEF7E1FE29463D
S3150800B7F02348FEF7B9FE94F8A430DBB2012B0CD02F
S3150800B80000F0E2FD1F4B1B685BB91F4B1B68A34288
S3150800B8100ED038BD1C4B1C68DFE7002384F8A43023
S3150800B820EEE700F0AFFDFFF7E7FB00F0CDFDECE734
S3150800B830144B1B68B3B1154B1B6843B14FF050034B
S3150800B84083F31188BFF36F8FBFF34F8FFEE74FF077
S3150800B850E0234FF08052C3F8042DBFF34F8FBFF398
S3150800B8606F8FD6E7064B1A68094B1B689A4203D1B5
S3150800B870054B00221A60CCE7FFF758FFC9E700BF5F
S3150800B880A40C0020940C002074110020780C0020D1
S3150800B890A00C002058B110B50C46094A1168183199
S3150800B8A0FEF76DFE01212046FFF702FD10BD4FF0A1
S3150800B8B0500383F31188BFF36F8FBFF34F8FFEE7F3
S3150800B8C07411002070B110B514460246114B1B685E
S3150800B8D08BB94FF0500383F31188BFF36F8FBFF313
S3150800B8E04F8FFEE74FF0500383F31188BFF36F8F36
S3150800B8F0BFF34F8FFEE7084B186841F0004181619E
S3150800B900196818311046FEF72FFE01212046FFF769
S3150800B910CFFC10BD780C00207411002038B570B12A
S3150800B9200D4614460A4A11681831FEF71DFE0CB179
S3150800B9304FF0FF3521462846FFF7BAFC38BD4FF0D1
S3150800B940500383F31188BFF36F8FBFF34F8FFEE762
S3150800B9507411002038B5C368DC6824B304F11805EF
S3150800B9602846FEF725FE184B1B682BBB251D2846C7
S3150800B970FEF71EFEE06A154B1B68984201D9134B69
S3150800B980186000EB80002946114B03EB8000FEF798
S3150800B990EBFDE26A0F4B1B68DB6A9A4211D901205C
S3150800B9A00D4B186038BD4FF0500383F31188BFF371
S3150800B9B06F8FBFF34F8FFEE729460848FEF7D4FD81
S3150800B9C0E7E70020EEE700BF780C0020980C00207F
S3150800B9D0140D0020741100208C0C0020D00C0020BF
S3150800B9E038B51C4B1B6843B94FF0500383F31188D5
S3150800B9F0BFF36F8FBFF34F8FFEE741F00041016041
S3150800BA00C468F4B1FEF7D4FD251D2846FEF7D0FD1F
S3150800BA10E06A114B1B68984201D90F4B186000EB7E
S3150800BA20800029460D4B03EB8000FEF79DFDE26A78
S3150800BA300B4B1B68DB6A9A4202D90A4B01221A6031
S3150800BA4038BD4FF0500383F31188BFF36F8FBFF3F0
S3150800BA504F8FFEE7780C0020980C0020140D00206C
S3150800BA60741100208C0C0020034B1B680360034BE9
S3150800BA701B684360704700BF880C00209C0C0020A0
S3150800BA80F8B5C8B10C460546F9B100F07BFC1B4B6E
S3150800BA9019686B68C81A2268B2F1FF3F26D0184E9B
S3150800BAA036682F68B74201D08B4224D9824215D80E
S3150800BAB00023236001241AE04FF0500383F3118812
S3150800BAC0BFF36F8FBFF34F8FFEE74FF0500383F33B
S3150800BAD01188BFF36F8FBFF34F8FFEE75B1A1344CE
S3150800BAE023602846FFF7C0FF002400E0002400F08A
S3150800BAF06BFC2046F8BD0124F9E700BF9C0C00202A
S3150800BB00880C0020014B01221A6070478C0C00201B
S3150800BB10014B1868704700BF74110020054B1B685D
S3150800BB2033B1054B1B680BB10020704702207047E4
S3150800BB3001207047940C0020780C002000283ED085
S3150800BB4038B50446C36A204A1268D26A93422ED28E
S3150800BB508269002A05DB1C4A1268D26AC2F13802D9
S3150800BB608261616903EB8303184A02EB83039942F6
S3150800BB7005D0154B1B68DB6AE362012038BD251D1D
S3150800BB802846FEF715FD104B1B68D86AE062104B75
S3150800BB901B68984201D90E4B186000EB80002946B5
S3150800BBA00A4B03EB8000FEF7DFFC0120E6E7C26CD8
S3150800BBB0054B1B68DB6A9A4203D30020DEE70020A8
S3150800BBC070470120DAE700BF74110020140D002029
S3150800BBD0980C002000283BD038B504461E4B1B683D
S3150800BBE0834208D04FF0500383F31188BFF36F8F59
S3150800BBF0BFF34F8FFEE7036D43B94FF0500383F34E
S3150800BC001188BFF36F8FBFF34F8FFEE7013B0365C4
S3150800BC10C16AC26C91421DD00BB1002038BD051D0A
S3150800BC202846FEF7C5FCE06CE062C0F13803A36164
S3150800BC300A4B1B68984201D9084B186000EB800034
S3150800BC402946074B03EB8000FEF78EFC0120E5E74B
S3150800BC50002070470020E1E774110020980C0020AE
S3150800BC60140D0020002846D038B50446036D43B9A4
S3150800BC704FF0500383F31188BFF36F8FBFF34F8FD5
S3150800BC80FEE7C26C8A4200D20A46E16A914201D0B6
S3150800BC90012B00D038BD184B1B68A34222D0E262A4
S3150800BCA0A369002B02DBC2F13802A261626901EBCB
S3150800BCB08101124B03EB81039A42EBD1251D2846DD
S3150800BCC0FEF776FCE06A0E4B1B68984201D90C4BCE
S3150800BCD0186000EB80002946084B03EB8000FEF74E
S3150800BCE043FCD7E74FF0500383F31188BFF36F8FF8
S3150800BCF0BFF34F8FFEE7704774110020140D002024
S3150800BD00980C0020044A136898691368DB6A12685D
S3150800BD10C3F138039361704774110020054B1B6803
S3150800BD2023B1044B1A68136D01331365014B186868
S3150800BD30704700BF74110020064B1A6813682BB9A8
S3150800BD400123036023B9D368186870470023F8E70E
S3150800BD50002070477812002008B5416000619142C2
S3150800BD600CD8D21A83699A4201D3012008BD011D55
S3150800BD70094B1868FEF703FC0020F7E79A4201D240
S3150800BD80994206D2011D054B1868FEF7F8FB0020FC
S3150800BD90ECE70120EAE700BF7412002078120020C1
S3150800BDA030B583B000F0EEFA114B1B681BB100F0FA
S3150800BDB00BFB03B030BD0F4D2846FEF7C7FB0E4CF4
S3150800BDC02046FEF7C3FB0D4B1D600D4B1C60002380
S3150800BDD000930C4B0C4A10210A20FEF7F7FC044B83
S3150800BDE018600028E3D00949FFF7C8F8DFE700BF65
S3150800BDF070120020901200207C1200207812002079
S3150800BE007412002078110020C8110020E4D0000820
S3150800BE102DE9F041079F41B94FF0500383F311888C
S3150800BE20BFF36F8FBFF34F8FFEE7064614461D46D6
S3150800BE3088468FB1FFF7B4FF3E60C7F81880FD61EA
S3150800BE40069B3B62381DFEF78CFB2CB197F8283011
S3150800BE5043F0040387F82830BDE8F08110B588B0B0
S3150800BE60FFF79EFF124B1B68CBB10024059406947E
S3150800BE7007AA06A905A8FEF703FA059B0293069BDF
S3150800BE800193022300932346079A0A490A48FFF7B3
S3150800BE904DFA0A4B186010B1012008B010BD4FF0DA
S3150800BEA0500383F31188BFF36F8FBFF34F8FFEE7FD
S3150800BEB070120020ECD000084DC200086C12002059
S3150800BEC02DE9F04182B00446884617461D462C20C7
S3150800BED000F010FC064658B1002380F8283001907F
S3150800BEE0089B00932B463A4641462046FFF790FFAB
S3150800BEF0304602B0BDE8F08110B584B084462C20E7
S3150800BF00039003982C2808D04FF0500383F3118828
S3150800BF10BFF36F8FBFF34F8FFEE70398079860B1A3
S3150800BF200220079C84F82800019406980090604631
S3150800BF30FFF76EFF079804B010BD4FF0500383F368
S3150800BF401188BFF36F8FBFF34F8FFEE7B8B19C46DA
S3150800BF5003461848006858B300B585B000910192A9
S3150800BF60029305291CDCFFF7D9FD022810D000230F
S3150800BF701A4669460F480068FEF796FC15E04FF02A
S3150800BF80500383F31188BFF36F8FBFF34F8FFEE71C
S3150800BF900023069A694607480068FEF785FC04E010
S3150800BFA0002362466946FEF789FD05B05DF804FB85
S3150800BFB0002070477012002070B582B01B4B1B68BA
S3150800BFC01A6862B3DB681E68DC68251D2846FEF71A
S3150800BFD0EFFA236A2046984794F8283013F0040F9E
S3150800BFE0ECD0A36933449E4207D263602461294694
S3150800BFF00E4B1868FEF7C3FAE0E7002100910B46DE
S3150800C00032462046FFF7A2FF0028D7D14FF050034B
S3150800C01083F31188BFF36F8FBFF34F8FFEE7044A90
S3150800C020106802490860136002B070BD78120020DB
S3150800C0307412002038B50546FFF744FA0446074B44
S3150800C0401B68834205D800232B60044B1C602046DE
S3150800C05038BDFFF7B1FF01232B60F6E76812002011
S3150800C06070B582B006460D4617490968C968CC6896
S3150800C070201DFEF79DFA94F828C01CF0040F08D17D
S3150800C0802CF0010C84F828C0236A2046984702B091
S3150800C09070BDA16933462A4631442046FFF75CFE47
S3150800C0A00028F1D0002100910B4632462046FFF7C2
S3150800C0B04DFF0028E8D14FF0500383F31188BFF3F2
S3150800C0C06F8FBFF34F8FFEE77812002070B582B0EE
S3150800C0D006460C46FFF7EEF901A8FFF7ABFF019BF2
S3150800C0E033BB0546E4B9B04213D22246711B124B44
S3150800C0F01868FEF757FFFFF777FAD8B94FF0E0232D
S3150800C1004FF08052C3F8042DBFF34F8FBFF36F8FE4
S3150800C11010E0FFF769FA29463046FFF7A1FF09E064
S3150800C120064A126812680AB90124DEE71C46DCE7EB
S3150800C130FFF75AFA02B070BD701200207412002080
S3150800C14010B588B002E0049B002B0FDA002204A980
S3150800C1503D4B1868FEF719FD002873D0049B002B89
S3150800C160F1DA07990698059B9847ECE7069C6369F8
S3150800C17013B1201DFEF71CFA03A8FFF75BFF049B0B
S3150800C180092BE3D8DFE803F0050505303750050528
S3150800C190303794F8283043F0010384F82830059B9B
S3150800C1A0A169024619442046FFF7D6FD0028CDD0DE
S3150800C1B0236A2046984794F8283013F0040FC5D010
S3150800C1C0A269002100910B46059802442046FFF714
S3150800C1D0BDFE0028BAD14FF0500383F31188BFF390
S3150800C1E06F8FBFF34F8FFEE794F8283023F00103D3
S3150800C1F084F82830AAE794F8283043F0010384F835
S3150800C20028300599A16131B103460246014420460A
S3150800C210FFF7A2FD9AE74FF0500383F31188BFF3A7
S3150800C2206F8FBFF34F8FFEE794F8283013F0020F95
S3150800C23004D023F0010384F8283087E7204600F06D
S3150800C240DBFA83E708B010BD7012002000B583B092
S3150800C25001A8FFF771FD0199FFF738FFFFF770FF97
S3150800C260F6E740B110B5044600F08CF8E46900F032
S3150800C270ABF8204610BD4FF0500383F31188BFF387
S3150800C2806F8FBFF34F8FFEE710B584B014461A467A
S3150800C2906FF001030093019002910394002369460D
S3150800C2A002480068FEF70AFC04B010BD70120020B0
S3150800C2B082B0002301930D4B1B68B3F1FF3F08D0F2
S3150800C2C04FF0500383F31188BFF36F8FBFF34F8F7F
S3150800C2D0FEE74FF0500383F31188BFF36F8FBFF368
S3150800C2E04F8F019B002BFCD002B07047C400002082
S3150800C2F008480068006880F308884FF0000080F35B
S3150800C300148862B661B6BFF34F8FBFF36F8F00DF35
S3150800C31000BF000008ED00E0DFF80C00016841F4FA
S3150800C320700101607047000088ED00E04FF08073EF
S3150800C33040F8043C21F0010140F8081C054B40F880
S3150800C3400C3C40F8202C6FF0020340F8243C44389B
S3150800C350704700BFB1C200080000000000000000DE
S3150800C360074B19680868B0E8F04F80F30988BFF3EF
S3150800C3706F8F4FF0000080F311887047AFF300808D
S3150800C380741100204FF0500383F31188BFF36F8FA9
S3150800C390BFF34F8F0B4A136801331360012B00D08C
S3150800C3A070474FF0E023D3F8043D13F0FF0FF7D0A2
S3150800C3B04FF0500383F31188BFF36F8FBFF34F8F8E
S3150800C3C0FEE700BFC4000020094B1B6843B94FF0C5
S3150800C3D0500383F31188BFF36F8FBFF34F8FFEE7C8
S3150800C3E0013B034A13600BB983F31188704700BFFA
S3150800C3F0C40000200000000000000000000000004B
S3150800C400EFF30980BFF36F8F154B1A681EF0100FF4
S3150800C41008BF20ED108A20E9F04F10602DE90900C9
S3150800C4204FF0500080F31188BFF34F8FBFF36F8F23
S3150800C430FFF77CF94FF0000080F3118809BC1968F2
S3150800C4400868B0E8F04F1EF0100F08BFB0EC108A6D
S3150800C45080F30988BFF36F8F704700BFAFF3008082
S3150800C4607411002008B54FF0500383F31188BFF309
S3150800C4706F8FBFF34F8FFFF72BF828B14FF0E023EC
S3150800C4804FF08052C3F8042D002383F3118808BDAA
S3150800C4904FF0E022002313619361054B1B680549A1
S3150800C4A0A1FB03139B09013B5361072313617047E3
S3150800C4B094000020D34D62104FF0E023D3F8002DEE
S3150800C4C03D4B9A421CD04FF0E023D3F8002D3B4B4E
S3150800C4D09A421ED030B583B0394B1A78D2B201923F
S3150800C4E0FF221A701B78DBB28DF803309DF80330F3
S3150800C4F003F05003334A1370334B07221A601BE0CC
S3150800C5004FF0500383F31188BFF36F8FBFF34F8F3C
S3150800C510FEE74FF0500383F31188BFF36F8FBFF325
S3150800C5204F8FFEE7284A1368013B13609DF80330D6
S3150800C5305B00DBB28DF803309DF8033013F0800FF3
S3150800C540F0D1214B1B68032B08D04FF0500383F31F
S3150800C5501188BFF36F8FBFF34F8FFEE71B021A4A8E
S3150800C560136003F4E0631360019BDBB2144A137093
S3150800C5704FF0E024D4F8203D43F47003C4F8203D7E
S3150800C580D4F8203D43F07043C4F8203DFFF780FF00
S3150800C59000250E4B1D60FFF7BFFED4F8343F43F06D
S3150800C5A04043C4F8343FFFF7A3FEFFF7BFF8FFF791
S3150800C5B07FFE284603B030BD71C20F4170C20F41DD
S3150800C5C000E400E0A8120020A4120020C400002005
S3150800C5D0EFF305830F2B0FD9114A9B5CDBB2114A87
S3150800C5E012789A4208D94FF0500383F31188BFF3A3
S3150800C5F06F8FBFF34F8FFEE74FF0E023D3F80C3D64
S3150800C60003F4E063084A1268934208D94FF05003CE
S3150800C61083F31188BFF36F8FBFF34F8FFEE7704721
S3150800C620F0E300E0A8120020A4120020124A12F03B
S3150800C630070F1ED0D11D21F00701C1F50043134491
S3150800C6400A460E480260002141601344083B23F065
S3150800C65007030B48036059601960991A5160136003
S3150800C660084B1960084B1960084B4FF000421A60D6
S3150800C67070474FF40043E4E7CC120020C4120020B0
S3150800C680C0120020B8120020BC120020AC120020F4
S3150800C690164B1A461B688342FBD3516802EB010C02
S3150800C6A0844509D0416800EB010C634509D0036055
S3150800C6B0904219D010607047406801445160104696
S3150800C6C0F0E710B40A4C2468A3420BD05B681944FF
S3150800C6D0416013681B680360904200D010605DF8E3
S3150800C6E0044B70470460F7E7704700BFC412002088
S3150800C6F0C012002038B50446FEF7DCFE384B1B682E
S3150800C700B3B1384B1B681C4250D1002C50D004F1F1
S3150800C710080214F0070F02D022F007020832002A96
S3150800C72055D0314B1B68934253D330490C6804E00B
S3150800C730FFF77CFFE5E721461C466368934202D271
S3150800C7402368002BF7D1264B1B68A34243D00D68FC
S3150800C750083523680B6063689B1A102B10D9A0183C
S3150800C76010F0070F08D04FF0500383F31188BFF37A
S3150800C7706F8FBFF34F8FFEE743606260FFF788FF56
S3150800C780626819490B689B1A0B60194909688B423C
S3150800C79001D217490B60134B1B68134363600023D0
S3150800C7A02360144A13680133136002E0002500E091
S3150800C7B00025FEF719FF15F0070F0ED04FF05003AE
S3150800C7C083F31188BFF36F8FBFF34F8FFEE7002502
S3150800C7D0EFE70025EDE70025EBE7284638BD00BF63
S3150800C7E0C0120020AC120020BC120020C412002087
S3150800C7F0B8120020B4120020002834D038B50446F8
S3150800C800A0F1080550F8043C174A1268134208D1EB
S3150800C8104FF0500383F31188BFF36F8FBFF34F8F29
S3150800C820FEE750F8081C41B14FF0500383F3118816
S3150800C830BFF36F8FBFF34F8FFEE723EA020340F87B
S3150800C840043CFEF737FE54F8041C084A13680B44E8
S3150800C85013602846FFF71CFF054A13680133136067
S3150800C860FEF7C2FE38BD7047AC120020BC1200208D
S3150800C870B0120020DFF834D0F8F7C2FC0C480D4996
S3150800C8800D4A002302E0D458C4500433C4188C421D
S3150800C890F9D30A4A0A4C002301E013600432A24283
S3150800C8A0FBD300F06FF8F8F735FAFEE70000012031
S3150800C8B0000000201801002008D1000818010020F7
S3150800C8C00C940020FEE702440346934200D17047C9
S3150800C8D003F8011BF9E70000294B1B68834270B572
S3150800C8E004464BD0C369ABB1DB686BB10025E3697D
S3150800C8F0DB68595900293BD10435802DF7D1E36906
S3150800C9002046D96800F072F8E369196811B1204623
S3150800C91000F06CF8616911B1204600F067F8E1692A
S3150800C92011B1204600F062F8216B11B1204600F0E3
S3150800C9305DF8616B11B1204600F058F8A16B11B192
S3150800C940204600F053F8A16C11B1204600F04EF8CD
S3150800C950616C11B1204600F049F8E16A11B1204630
S3150800C96000F044F8236A4BB12046BDE870401847EA
S3150800C9700E68204600F03AF83146BBE770BD00BFA6
S3150800C980C800002070B50D4D0D4C641BA410002680
S3150800C990A64209D10B4D0C4C00F07EF8641BA4107E
S3150800C9A00026A64205D170BD55F8043B98470136C6
S3150800C9B0EEE755F8043B98470136F2E7F8D0000849
S3150800C9C0F8D00008F8D00008FCD000087047704777
S3150800C9D00A44914200F1FF3300D1704710B511F8AF
S3150800C9E0014B03F8014F9142F9D110BD38B5054600
S3150800C9F0002941D051F8043C0C1F002BB8BFE4189D
S3150800CA0000F03EF81D4A136833B96360146028467F
S3150800CA10BDE8384000F03AB8A34208D92068211882
S3150800CA208B4201BF19685B6809182160EDE71A4651
S3150800CA305B680BB1A342FAD911685018A0420BD112
S3150800CA4020680144501883421160E0D118685B6879
S3150800CA50536008441060DAE702D90C232B60D6E746
S3150800CA60206821188B4204BF19685B68636004BF9D
S3150800CA70091821605460CAE738BD00BF0894002031
S3150800CA800148FFF7A3BF00BF049400200148FFF741
S3150800CA909EBF00BF04940020F8B500BFF8BC08BCD0
S3150800CAA09E467047F8B500BFF8BC08BC9E4670475E
S3150800CAB0494E49545F54687265616400B0CA0008FB
S3150800CAC00000000000000000000000000000000058
S3150800CAD0000400002F000000000000000000000015
S3150800CAE04D41494E5F5761746368646F6700000083
S3150800CAF04D41494E5F55706461746554696D657240
S3150800CB00000000004D41494E5F4576656E745F46EC
S3150800CB106C616773000000004D41494E5F43414E0A
S3150800CB205F52785F51756575650000004D41494E45
S3150800CB305F54687265616400E0CA0008000000007E
S3150800CB400000000000000000F0CA00080000000015
S3150800CB50000000000000000004CB000800000000F0
S3150800CB60000000000000000018CB000800000000CC
S3150800CB7000000000000000000000000000000000A7
S3150800CB802CCB000800000000000000000000000098
S3150800CB900000000000040000210000000000000062
S3150800CBA0000000005045434F5F4576656E745F464A
S3150800CBB06C616773000000005045434F5F55706411
S3150800CBC061746554696D6572000000005045434FF5
S3150800CBD05F54687265616400A4CB00080000000019
S3150800CBE00000000000000000B8CB000800000000AC
S3150800CBF00000000000000000CCCB00080000000088
S3150800CC000000000000000000000000000004000012
S3150800CC1028000000000000000000000056415248AD
S3150800CC205F4D7574657800001CCC00080300000091
S3150800CC3000000000000000000000000001000000E5
S3150800CC4000000000010000000100000000000000D4
S3150800CC500000A0C0000040411100000000000000D4
S3150800CC60000000000000C84211000000000000009B
S3150800CC70000000000000C84211000000000000008B
S3150800CC80000000000000C842010000000000B84192
S3150800CC90000020C2000048421100000000002041A8
S3150800CCA0000000000000404111000000000000C024
S3150800CCB0000000C00000000009000000000000009D
S3150800CCC0000070C20000C842090000000000000011
S3150800CCD0000070C20000C842090000000000000001
S3150800CCE0000048C200008C42090000000000000055
S3150800CCF00000A0C00000604109000000000000001C
S3150800CD00000020C1000020410900000000000000CA
S3150800CD10000000000000A04009000000000000001C
S3150800CD20000048C200001643090000000000000089
S3150800CD300000A0410000F0410900000000000000CA
S3150800CD40000000000000A0400900000000000000EC
S3150800CD500000000000001643080000000000000064
S3150800CD6000000000010000000800000000000000AC
S3150800CD7000000000FFFFFFFF11000000333353409F
S3150800CD800200000000008040414443445F4D757432
S3150800CD906578000088CD0008030000000000000048
S3150800CDA000000000414E50495F4D757465780000DB
S3150800CDB0414E50495F4576656E745F466C61677390
S3150800CDC000000000414E50495F5468726561640076
S3150800CDD0A4CD0008030000000000000000000000C9
S3150800CDE0B0CD0008000000000000000000000000B0
S3150800CDF0C4CD00080000000000000000000000008C
S3150800CE000000000000040000100000000000000000
S3150800CE100000000000000000000004419A996D41DE
S3150800CE2000000441000020410000A040000020410D
S3150800CE300000A040414E504F5F4576656E745F46D0
S3150800CE406C61677300000000414E504F5F55706477
S3150800CE5061746554696D657200000000414E504F5B
S3150800CE605F5468726561640034CE000800000000F3
S3150800CE70000000000000000048CE00080000000086
S3150800CE8000000000000000005CCE00080000000062
S3150800CE900000000000000000000000000004000080
S3150800CEA01800000000000000000000000004004810
S3150800CEB04000000001000000000000000100000022
S3150800CEC00000000001000000000000000004004807
S3150800CED02000000001000000000000000100000022
S3150800CEE000000000010000000000000000080048E3
S3150800CEF000400000010000000000000001000000E2
S3150800CF0000000000000000000100000000000048CA
S3150800CF100001000001000000000000000100000000
S3150800CF2000000000000000000100000000040048A6
S3150800CF308000000000000000000000000100000062
S3150800CF400000000000000000010000000008004882
S3150800CF500080000000000000000000000100000042
S3150800CF600000000000000000010000000004004866
S3150800CF70080000000000000000000000010000009A
S3150800CF800000000000000000010000000004004846
S3150800CF901000000000000000000000000100000072
S3150800CFA0000000000000000001000000000000482A
S3150800CFB000800000000000000000000001000000E2
S3150800CFC0000000000000000001000000000300202F
S3150800CFD00000000014D00008010000000200000054
S3150800CFE0535049445F4576656E745F466C61677356
S3150800CFF000000000535049445F4144435F4D757437
S3150800D00065780000E0CF000800000000000000007E
S3150800D01000000000F4CF0008030000000000000034
S3150800D0200000000054454D505F5468726561640005
S3150800D03024D00008000000000000000000000000E6
S3150800D04000000000000400001800000000000000B6
S3150800D050000000005553464C5F4D75746578000016
S3150800D06054D0000803000000000000000000000083
S3150800D07044656661756C740070D000080000000095
S3150800D0800000000000000000000000000002000090
S3150800D090180000000000000000000000A086010043
S3150800D0A0400D0300801A060000350C0040420F00B0
S3150800D0B080841E0000093D0000127A000024F40056
S3150800D0C000366E010048E801006CDC020000000032
S3150800D0D000000000010203040607080949444C45FC
S3150800D0E000000000546D725100000000546D72205B
S30D0800D0F05376630000000000FE
S30D0800D0F8B5290008000000003C
S30D0800D100912900080000000057
S3150800D10800FF0000080200201002002000000000AE
S3150800D11800000000000000000000000000000000F9
S3150800D12800000000000000000000000000000000E9
S3150800D13800000000000000000000000000000000D9
S3150800D148000000000060000000000000E0E90000A0
S3150800D15800000000000000000100000000000000B8
S3150800D1680100000001000000000000000040000067
S3150800D1780000000000E800000000000000000000B1
S3150800D1880000000000000000010000000100000087
S3150800D1980000000000093D00010000001000000022
S3150800D1A80000000000000000000000000000000069
S3150800D1B80100000000000000000000000000000058
S3150800D1C820000000AAAAAAAACC0000200000000095
S3150800D1D8CC920020349300209C9300200000000085
S3150800D1E80000000000000000000000000000000029
S3150800D1F80000000000000000000000000000000019
S3150800D2080000000000000000000000000000000008
S30D0800D218000000000000000000
S7050800C875B5
